:020000041000EA
:1000000000B5324B212058609868022188439860DF
:10001000D860186158612E4B002199600221596106
:100020000121F02299502B49196001219960352056
:1000300000F044F80222904214D00621196600F024
:1000400034F8196E01211966002018661A6600F04E
:100050002CF8196E196E196E052000F02FF8012189
:100060000842F9D1002199601B49196000215960AB
:100070001A491B48016001219960EB211966A021F2
:10008000196600F012F800219960164914480160C1
:100090000121996001BC002800D000471248134993
:1000A000086003C880F30888084703B5996A0420EC
:1000B0000142FBD001200142F8D103BD02B5186610
:1000C0001866FFF7F2FF186E186E02BD00000240BE
:1000D000000000180000070000035F00212200005C
:1000E000F4000018222000A00001001008ED00E03C
:1000F00000000000000000000000000074B24E7A12
:1001000000200420F7010010CB010010CD010010E9
:10011000C9010010C9010010C9010010C901001077
:10012000C9010010C9010010C9010010CF01001061
:10013000C9010010C9010010D1010010D301001045
:10014000C1010010C1010010C1010010C101001067
:10015000C1010010C1010010C1010010C101001057
:10016000C1010010C1010010C1010010C101001047
:10017000C1010010C1010010C1010010C101001037
:10018000C1010010C1010010C1010010C101001027
:10019000C1010010C1010010C1010010C101001017
:1001A000C1010010C1010010C1010010C101001007
:1001B000C1010010C1010010C1010010C1010010F7
:1001C000EFF30580103800BE00BE00BE00BE00BECA
:1001D00000BE00BEF2EB887194890010B489001053
:1001E0003802001090A31AE71E481F49086006C88D
:1001F00081F3088810471D480068002801D019487D
:10020000F3E70DA40ECC002902D000F012F8F9E7B4
:100210001749184A002000E001C19142FCD116495B
:100220008847164988471649884700BEFDE701C937
:1002300001C29A42FBD37047B4890010C00000206D
:1002400020160020149F001000000420000004204D
:10025000149F001000100420001004200000000073
:10026000704700000000000008ED00E0000000D032
:10027000201600202C2800203D430010F904001017
:1002800035430010F8B5C0460448054B10B583420D
:1002900003D0044B002B00D0984710BD201600203F
:1002A000201600200000000006480749091A8B109C
:1002B000C90FC91810B5491003D0044B002B00D04A
:1002C000984710BD201600202016002000000000D6
:1002D00010B5074C2378002B09D1FFF7D5FF054B4C
:1002E000002B02D0044800E000BF0123237010BDA2
:1002F000A81900200000000028810010054B10B54F
:10030000002B03D00449054800E000BFFFF7CCFFF5
:1003100010BDC04600000000AC190020288100106C
:10032000F0B5DE464E4645465746E0B593B01E1C36
:100330001C9B041C684890469A46894604F00CFAB7
:10034000201C02F0B7FA0400301C0D0002F0B2FAD3
:100350000A900B91504602F0ADFA0A9A0B9B089056
:1003600009911D980692079302F0A4FA0490059152
:10037000404602F09FFA02900391484602F09AFA32
:10038000564E0090019122002B00300004F068FAD4
:1003900040461D9902F088FA002800D199E0504AA1
:1003A000504B2000290001F044FE4E4B0C900D9163
:1003B0000A980B994A4A01F03CFE002310934A4BDD
:1003C0000E900F911193494B9B46504602F072FAE2
:1003D0000C9A0D9B01F006FE01F0E2FE824602F04F
:1003E00069FA3F4A3F4B06000F0001F022FE04006D
:1003F00040460D0002F05EFA02000B0020002900CA
:1004000001F0F0FD01F0CCFE8046484602F052FAC1
:100410000E9A0F9B01F0E6FD01F0C2FE8146109896
:1004200002F048FA0A9A0B9B040040460492059396
:100430000D000696079702F03DFA02900391484698
:1004400002F038FA2200009001912B00119804F07C
:1004500007FA5B461B68986807F0F0FC012000F083
:10046000D1FE1F4A1F4B2000290001F0BBFD01F007
:1004700097FE414610901D9802F010FA0028A4D172
:100480001B4804F069F9484602F014FA0400109879
:100490000D0002F00FFA06900791504602F00AFA9A
:1004A0000A9A0B9B0490059140460292039302F036
:1004B00001FA104E0090019122002B00300004F050
:1004C000CFF9002013B0F0BCBB46B246A946A04607
:1004D000F0BD00231093D3E728810010488100105D
:1004E000FCA9F1D24D62503F80810010A81000207D
:1004F000B4810010D0810010F0B5DE4657464E465C
:100500004546E0B583B004F099F8FA20800000F089
:1005100079FE364B364F9B46364B374E9A46374B15
:10052000374D9946374B384C9846584604F014F9E5
:10053000504604F011F9484604F00EF9404604F024
:100540000BF9380004F008F9300004F005F9280030
:1005500004F002F9200004F0FFF804F073F86328B7
:100560001CD00CDC312831D0322829D1274804F0A6
:10057000F3F8274804F0F0F804F064F8D5E76828A9
:1005800015D078281CD1234804F06AF9002003B064
:10059000F0BCBB46B246A946A046F0BD1E4804F0DA
:1005A000DBF81B4804F0D8F804F04CF8BDE71B4812
:1005B00004F0D2F8164804F0CFF804F043F8B4E79A
:1005C000174B0100180004F04BF9AEE70021FE22A2
:1005D000144B019100939205134B1448FFF7A0FEB2
:1005E0000B4804F0B9F804F02DF89EE708820010DB
:1005F0009882001034820010A882001054820010EB
:10060000B482001080820010C0820010EC820010C2
:10061000CC8200102483001014830010FC82001090
:10062000648300100000A04100002042C3F51CC1FB
:100630008023DB051868000F7047C0460FB400B573
:10064000084883B004F088F8049B002B07D005A964
:100650001800019103F00EFE034804F07DF801201C
:1006600003F020FE788300108883001070B5EFF34C
:10067000108C72B60D4D2B68002BFCD0BFF35F8F32
:100680000724CB08C618C05C01230C40A3401C0003
:100690000440034207D118433070BFF35F8F2C60D2
:1006A0008CF3108870BD1000FFF7C8FF2C0100D03C
:1006B000F8B54746CE46884680B5EFF3108C72B643
:1006C0001C4D2C68002CFCD0BFF35F8F9A4222D8BF
:1006D00007210126894602E00132934218D34D4694
:1006E00037001540AF40D4080119045D2742F3D10B
:1006F00010003C430C70BFF35F8F00220D4B1A605B
:100700008CF3108800280EDBC0BCB946B046F8BD9B
:1007100001204042EFE7BFF35F8F00232B608CF393
:100720001088012040424346002BEDD00898FFF787
:1007300085FFC0462C0100D0044A1078431CDBB270
:10074000172B00D9102313707047C046E00F00200C
:1007500010B5064B064C82B00100009318221F23EF
:100760002000FFF7A5FF02B010BDC0468C8300102B
:100770006C2300200021044B044ABFF35F8F02C3A7
:100780009342FAD17047C046000100D0800100D0EA
:10079000054B064A1360064A136053609360D360AA
:1007A00013615361936170478080808000E400E0B2
:1007B00004E400E01F2318401E3B8340002905D0BD
:1007C000C021044A490053501360704780220149F8
:1007D0008B50FAE700E100E001228240034B1B68E6
:1007E00013405A1E9341D8B27047C04600E100E062
:1007F00001238340014A13607047C04600E200E0D5
:10080000064B10309B688000C358054A00209B1A95
:100810002F229A424041C0B27047C04600ED00E02E
:10082000E40F002070B50D00EFF3108672B60F4A8A
:100830001368002BFCD0BFF35F8F0D4B10309B680B
:1008400084001B590B4A934203D09D4201D001F012
:1008500033F8074B9B681D51BFF35F8FBFF35F8F6A
:100860000022024B1A6086F3108870BD240100D06C
:1008700000ED00E0C1010010F0B557464E46DE46DF
:100880004546E0B585B0060000911700EFF3108BE8
:1008900072B66A4A1368002BFCD0BFF35F8F002545
:1008A000674B5D579A46002D00DAA9E06B00654C56
:1008B00001935B199B009846A146C1444B465246A2
:1008C0009B7910361370604BB6009B6899590B1BCF
:1008D0002F2B33D95D4B994200D0ACE0019B4246AF
:1008E0009C465B4B6544AD0063535A4B0232A218E1
:1008F000043B9B1A1B05584A5B0D651913436B801B
:10090000564B0121AB80FF23AB71009BEF71AB60B5
:100910004B460B4319004C4B9B689951BFF35F8FBB
:10092000BFF35F8F0022454B1A608BF3108805B030
:10093000F0BCBB46B246A946A046F0BD01200A0065
:100940008243D3798C46BB4231D845461300444993
:100950001B1B5B415943090D3D4B63533D4B023516
:100960006519043B5B1B1B053B4D5B0D2B43AA46E6
:100970004D466B800425AC465546E044131F444465
:100980001B1B1B055B0D1D434B46997100999D80F8
:1009900099604946DF71334B01431360BBE7580050
:1009A000C01880002018C179B9422FD9020006234F
:1009B000D356002BF3DA02932B4B61460393131D9E
:1009C0009A4604235B429C46E14450464B461B1A20
:1009D0001B055B0D9C46204B95719846634640462F
:1009E00003439380019B5A199200039BA418A38090
:1009F000029B1C4AA371009B2260E771A3608AE7F7
:100A000000F05AFF002553465D574FE79088029348
:100A10004005131D9A46031561469C464046D44442
:100A2000634604302018181AE0230005400D1B020D
:100A300018430390C5E700F03FFF4FE7240100D0C3
:100A400025280020E40F002000ED00E0C101001087
:100A500000A1FFFF1410002000E0FFFF01BDFFFF19
:100A6000AAAA00000148804701BD000070B501241A
:100A70000443EFF30581EFF3108C72B6214A13683B
:100A8000002BFCD0BFF35F8F1F4B05001F4AED1AF0
:100A90006D416A43120D1E4D8900AE6852B2765800
:100AA000A6421CD00621595691421CD012215956FB
:100AB000914222D01E215956914220D02A215956C6
:100AC0000324914210D0134B19781A708171BFF32F
:100AD0005F8F00220B4B1A608CF3108870BDAB68DF
:100AE0000D4C5C50EFE700246100091989005B1888
:100AF000FF21997109499980E5E70124F4E702246F
:100B0000F2E7C046240100D0E40F0020AAAA0000AA
:100B100000ED00E025280020C101001001BDFFFF0D
:100B200010B5084B084C82B0010000930022052349
:100B30002000FFF7BDFD002801DB1F23181A02B0BB
:100B400010BDC046A883001029280020024B9C46F7
:100B500061448900016070474000003470B5114C59
:100B6000114DAC420FD2FF262368002B0CD0FFF7AB
:100B7000E3FD01002000FFF7E9FFA680BFF35F8FD0
:100B80000834AC42F0D370BDFFF7D6FD0100200061
:100B9000FFF7DCFF2671BFF35F8F0834AC42E3D36D
:100BA000F1E7C046101600202016002010B5040002
:100BB000FFF7C2FD01002000FFF7C8FFFF232371EC
:100BC000BFF35F8F10BDC04610B504000120FFF7D2
:100BD000BFFD034BC3189B002360BFF35F8F10BDA5
:100BE00040000034034B9C46614489000160BFF320
:100BF0005F8F7047400000340A4B1968EFF3108094
:100C000072B60A68002AFCD0BFF35F8F1B68BFF37F
:100C10005F8F00221A6080F3108840BF00200021FF
:100C20007047C04604280020F0B5DE4657464E46C1
:100C30004546E0B587B0EFF30583032201251A404E
:100C4000954091008846A946B34B03925C58B34B3C
:100C50001D60B34B04934B46B24843630823E55EE3
:100C6000002D37DAA3881BB2002B00DBADE0A3799F
:100C7000002B00D0EEE00823E05E002820DB4300DC
:100C800062691B18DB00D3189E68DD68731C00D1F5
:100C900011E1A44801004144826A0B69B71A9B1A0A
:100CA0009F4215D30123026A039883401A420FD052
:100CB0009C4800F0B5FB8D4202DCCCD18642CAD9FB
:100CC00040BF07B0F0BCBB46B246A946A046F0BD47
:100CD0000E61EDE762696B0092465B19DB009A4496
:100CE00053469E68DF6800F09BFB8F42BADC00D160
:100CF00003E1002F00DAE8E05246534652691B69CF
:100D00009346049A934200D1D9E052460821605E8E
:100D10005288000459461043984700900191009969
:100D2000019A0B001000134300D1CEE013000A001B
:100D3000B61A9F41002806DB7A4800F071FB009E3E
:100D4000019F36184F4153469E60DF6000229A5E35
:100D5000002A00DA86E7530099186069C900411833
:100D600002938B68C9689B46B94200DD7AE702D1DD
:100D7000B34200D976E708239C46A444059565460E
:100D80002281A446029B2C0006E053009918C9005A
:100D900041188D68C968AB469B18DB00C318B9427F
:100DA00006DC00D1B3E01C000023E25E002AECDA8E
:100DB000230064469C4653461A806346059D1D8069
:100DC000A3881BB2002B00DA51E72269EFF31081F0
:100DD00072B61368002BFCD0BFF35F8F0123A78886
:100DE0005B42A3803FB22369BFF35F8F00221A608A
:100DF00081F31088002F00DA39E72300083322003E
:100E00009A4666697B00DB19DB00F3189968504647
:100E10008C460824115FDD68002910DB029306E090
:100E2000AB4244D00023E15E2000002906DB4C00E9
:100E30006418E4003419E368AB42F1DD029B0780DB
:100E400000201F5E1980002FDCDA1400A379002B2C
:100E500000D110E70023A37126000823E15E0836C5
:100E60004B1C00D12CE70800A246656902E03E0059
:100E70004B1C1AD04B005B18DB00EF180A008C46A5
:100E8000E95E7B881BB2002BF1DA01235B42DC17A1
:100E9000BB60FC60824205D0534631801B893B8099
:100EA00053461A8160464B1CE4D15446E5E6A368DC
:100EB0006345B7D9C2E76B1C00D0EAE6F8E65B46AB
:100EC00058461B69984700281BD153461B88226946
:100ED0002381EFF3108372B611680029FCD0BFF3B1
:100EE0005F8F514662880A8022696580BFF35F8FF9
:100EF0000021116083F31088B4E6864200D8F8E63A
:100F0000B0E65B461A685B680092019307E7B34559
:100F100000D848E74CE7C046E82700203C70054071
:100F2000290C00100040054070B52E4C2569002D9D
:100F300004D00A212C48FFF709FE70BD2B4E032177
:100F4000300000F063FAE660FFF7F6FB284B03225F
:100F50009C46D02322701B061B6801216370254B21
:100F60006044A3600F2380002061022063806369D6
:100F70004942A18019800231198647311D83585298
:100F800018315A5275325C399952183201319952DE
:100F900018320131995218320131995208351832FC
:100FA0009D52023118329952183201319952183239
:100FB0000131995218320131995218320131995246
:100FC0001832013199520C4B0C49DC60013035620A
:100FD000FFF728FC01210320FFF7ECFB084B1D6005
:100FE000A7E7C0462C100020042800200040054040
:100FF00040000034FFFF1000E8270020290C0010FB
:1010000038600540004870472C100020F8B51F00DC
:1010100008AB1B7804001600002B08D100F008FA7A
:1010200032003B00121A8B41002B00DA52E0226999
:10103000EFF3108072B61368002BFCD0BFF35F8F04
:101040000223E15E63694A005218D2009B182269AC
:10105000002936DB1D886580BFF35F8F0025156092
:1010600080F31088069A9E60DF601A61079A5A61C1
:101070005A8801325204520C101C002A1FD082B22E
:101080005880080410432669EFF3108772B632685F
:10109000002AFCD0BFF35F8FA2881A80A180236949
:1010A000BFF35F8F00221A6087F310880A49237804
:1010B0008C4601329A40E36863441A60F8BD01200F
:1010C000DDE7BFF35F8F0023136080F310880120FA
:1010D0004042F3E70020F1E73C20000070B501003A
:1010E0000469EFF3108C72B620680028FCD0BFF3BF
:1010F0005F8F02200D5E4C6968004019C000241803
:101100000869002D36DB26884E80BFF35F8F0026EE
:1011100006608CF31088E3606388049801332061D3
:101120005B0405985B0CA26060611A1C002B1FD049
:1011300093B22804628018430A69EFF3108C72B6E8
:101140001368002BFCD0BFF35F8F8B8823808D80CA
:101150000B69BFF35F8F00221A608CF310880B7845
:1011600001329A40CB6808498C4663441A6070BDCE
:101170000122DDE7BFF35F8F002303608CF310884B
:1011800001204042F3E7C0463C20000010B54389EF
:101190000A1493421ADD53009B184269DB00D318EE
:1011A0000469EFF3108C72B62268002AFCD0BFF3FA
:1011B0005F8F5A88090494B2090C8A4208D00369E7
:1011C000BFF35F8F00221A608CF31088002010BDDF
:1011D0008022120214435C80012302698371BFF3F1
:1011E0005F8F002111608CF31088044902788C46CF
:1011F0009340C268012062441360E8E73C2000008D
:1012000040787047F0B5C64600B582B0040000F0E3
:101210000FF9FA2206000F0020000023002192009F
:1012200001F0FAFA8019794104000D1E02DA012456
:101230002E4D644206267642F71736196F41AF42AB
:1012400014D811D000F0F4F832003B00121A8B4190
:10125000002B15DC002B46D02000290000F026F9D9
:1012600002B080BCB846F0BDA642EBD900260027EC
:1012700000F0DEF832003B00121A8B41002BE9DD52
:1012800000F0D6F832003B00121A8B41002B0ADB2B
:1012900000230193164B3200009316483B00FFF7E2
:1012A0001DFF0130D8D000233900B0469C46124AB9
:1012B0001248536A994204D8966A4645CCD299425C
:1012C000CAD10668EFF3108772B63368002BFCD0E2
:1012D000BFF35F8F0368BFF35F8F66461E6087F3BF
:1012E000108820BFE5E7002AB6D0C9E7FFFFFF7FDF
:1012F000F90B00102C1000200040054004280020AD
:10130000F0B557464E46DE464546E0B506000F00AE
:1013100085B0EFF3058399468B46002B12D03849F0
:1013200000204B6ABB4206D38A6ADB1B591E8B41E5
:10133000B2424041184305B0F0BCBB46B246A94694
:10134000A046F0BD2F4B9A46DB68984653461B7863
:101350004046039300F064F84246039B04000433C4
:101360009B009B580D001B1A39003000001BA9413F
:10137000894510DC0DD020BF214A0020536A5B450F
:10138000D9D3926ADB1B591E8B41B24240411843AC
:10139000D1E78342EFD900F04BF832003B00121A3C
:1013A0008B41002B1ADB00230193174B3200009373
:1013B00050463B00FFF792FE011E0FDD104B5A6AAC
:1013C0005A451BD39B6AB34216D35046FFF7DEFE45
:1013D0000B4A0020536A5B45ADD3D2E7084A002090
:1013E000536A5B45A7D30020926ADB1BB24240419F
:1013F0005A1E934118439EE75A45E6D120BFE4E7C1
:10140000004005402C100020F90B001010B5024AD6
:101410000248FFF72BF910BDC48300107023002091
:101420000300416A0A00986A596A8A42FAD17047F1
:10143000034B596A0A00986A596A9142FAD1704777
:101440000040054070B504000D00174A536A1900AA
:10145000966A536A8B42FAD13000190024184D4124
:10146000AB4216D813D0104B2A005B6A9D4203D9B9
:101470000D494B6A9342FCD3934207D10A4A02E0DA
:10148000516A994202D1916AA142F9D370BDA64234
:10149000E9D9054B5B6A1C005A1CEFD001220124DC
:1014A0006442E5175242E3E700400540064A536AAA
:1014B0009942FCD807D1044B02E05A6A914202D10A
:1014C0009A6A9042F9D8704700400540F8B5DE4668
:1014D0004E4657464546E0B58B4605000A9918002A
:1014E000160000F03BFB0A9B6C001F02324B641994
:1014F0009C46A4006444636881469F4200D96760AB
:101500002B1FDBB29846012B30D9C02380229B01D0
:10151000E31812011A60294BAD0059599A46002967
:101520001BD17301E026226853401E4080234246AF
:101530005B01E3181E60012A30D9802380229B01C1
:10154000E31812011A6053464A4667605A51F0BCCC
:10155000BB46B246A946A046F8BD586900F0FEFA5F
:10156000013043001B18033BFDD2DAE75B46012B39
:10157000CBD1C02303229B01E3181A60023AA3686F
:101580001A42FCD07301E0262268AD0053401E4091
:1015900080230A4A5B019246E3181E605A4621687E
:1015A000514003220A401A6001225B469A40A36818
:1015B0001A42FCD0C1E7C0460080004074230020DE
:1015C000F0B546464F46D646C0B51F00344B4400E2
:1015D0009C462418A4006444636888461600FF2BC8
:1015E00002D880235B006360031FDBB29A46012BA5
:1015F00030D9C02380229B01E31812011A60294BC5
:1016000085005959994600291BD17301E0262268AB
:1016100053401E40802352465B01E3181E60012A9E
:1016200030D9802380229B01E31812011A608023A5
:101630005B0063604B465F51E0BCBA46B146A846CA
:10164000F0BD586900F08AFA013043001B18033BD3
:10165000FDD2DAE74346012BCBD1C02303229B0105
:10166000E3181A60023AA3681A42FCD07301E0261C
:101670002268850053401E4080230A4A5B01914640
:10168000E3181E6042462168514003220A401A6056
:10169000012342469340A2681342FCD0C1E7C046F2
:1016A0000080004074230020014B8000C058704728
:1016B00074230020F8B5040021481E0017000D0017
:1016C00000F04CFA0100380000F048FA069B36049E
:1016D0001B031E432368002B20DB1A4B1A49E31817
:1016E0005A1E93418022920194465B421B0B174A7B
:1016F0001B0363441360164A13601F000A68974374
:10170000FBD1144B2560E2182123A06013602368ED
:10171000002BFCDA0823E6601360F8BD3F23226843
:101720001340AB42D9D1A3681B051B0D8342D4D112
:10173000EE22E368D2021340B342CED1EDE7C046B9
:10174000001BB7000040FDBF08C0004000E00040A3
:1017500000F000400430000010B580241C4BE4056C
:101760001C6000281AD001231A4C18431A4BDC6164
:101770001A4C44401C62596298628021144BC9057E
:101780001960174817490860E021C9041960002A48
:1017900007D18022144B12061A6010BD0E4BD8617F
:1017A000EBE753019B1A9B009A18802312015B04FC
:1017B0009A4209D213000D490B60074B5A608022F0
:1017C000094BD2051A60E8E7094B1A00F3E7C04657
:1017D00000B00540D3C007B0008005402D3FF84F52
:1017E000FCFF01000820014000A00540D827002090
:1017F000FFFFFF008023024A9B000B43D362704728
:1018000000800540002310B50100988A1B8B984783
:1018100010BDC046162310B50100188802331B887E
:10182000984710BDF8B54746CE4680B50F1E18D074
:1018300014239946043304000025012698464B469C
:101840001888434621681B88984701C4431E984165
:1018500001350640AF42F2D13000C0BCB946B046B7
:10186000F8BD0126F8E7C046002370B504000D005E
:10187000988A05491B8B984703000020002C01DB48
:101880000130A0402900984755420000AA23064A8B
:101890001B0113608D235B00D3600449044B196066
:1018A0005368002BFCDA70470040024000B0FA0099
:1018B000006002407047C04610B50148FEF7BEFE0A
:1018C000E883001070B5074D074EB54209D20024D9
:1018D000013E761BB60808CD984723000134B34279
:1018E000F9D170BDE08000101C810010054B064A44
:1018F00006491A60064A074B1A6010000B689843A5
:10190000FBD1704700E00040BFCDFBFE08C00040A7
:10191000FE7F3C0000F00040044BDB6C002B03D149
:101920008022034BD2021A607047C046000011505B
:101930004C201150044A054B1A60054A1368DB011C
:101940008033FBD17047C046FFFFFF0100F000402D
:1019500008C000404022034B9A675A671A67DA664C
:101960007047C04600F0014010B5FEF703FF10BD00
:10197000F8B52749274C284D641AA6103200302E9E
:1019800000D930222800920001F00CF8BC2C3BD882
:1019900030202F232C196407204A801BE40F9B1B47
:1019A000052B16D93700002C02D0B300771CEA5063
:1019B000001B33199B004108EB18C900C9181A60B5
:1019C0005A6008339942FAD1012303421CD098434C
:1019D000C619B300EA50731C2F2E15D09B00EA5095
:1019E000B31C2E2E10D09B00EA50F31C2D2E0BD0D2
:1019F0009B00EA50331D2C2E06D09B00EA50731D2D
:101A00002B2E01D09B00EA50054B9D60F8BDC046CF
:101A100000010010C001001000000020C1010010F2
:101A200000ED00E0002310B5294C82B0A367FFF75A
:101A30002DFF0122274B1A60636C012BFCD103227E
:101A4000254B1A60224A936B012BFCD10133009382
:101A50000121224A22480433FFF72CFE05230121ED
:101A60000093204A2048FFF725FE0022022104208F
:101A70001E4BFFF7A5FD0022012105201C4BFFF79F
:101A80009FFD0022002107201A4BFFF799FD00223D
:101A900000210820174BFFF793FD8023DB00009304
:101AA000002200210920134BFFF710FD0022104BEC
:101AB00000210620FFF784FD0420FFF7F5FD0E4905
:101AC00000F04CF801000020FFF794FE02B010BDBA
:101AD000008000403CB0004030B00040002F68590A
:101AE00000800240008C864700C00240001BB70007
:101AF00040597307006CDC0240420F00014804218A
:101B0000014B18475010002025180010124A936FFF
:101B10009B0815D29066D166002905D0FFE7FFE744
:101B2000FFE7516F106F704704B580210906C21797
:101B30005140002800D0C84306F092FA002104BDAD
:101B4000F0B5146E556E576F166FFFF7E3FF14660E
:101B5000556657671667F0BD000000D0114A936FB5
:101B60009B0813D210665166002905D0FFE7FFE7F6
:101B7000FFE7516F106F704704B5002801D00020B7
:101B8000C04306F06DFA002104BDC046F0B5146EE6
:101B9000556E576F166FFFF7E5FF1466556657676A
:101BA0001667F0BD000000D094464A4A926F920832
:101BB000624601D228E0C046F0B5464E346E756EDE
:101BC000776F366F00F020F89446424A14665566E7
:101BD000576716676246F0BD94463E4A926F920878
:101BE000624601D254E0C046F0B53A4E346E756E8E
:101BF000776F366F00F04CF89446364A1466556697
:101C0000576716676246F0BD002B24DB11D0002910
:101C10003EDA00B5C943404200D1013100F038F846
:101C2000C943404200D10131DB43524200D101336C
:101C300000BD002AEBD1002801D1002905D00020E9
:101C4000C90FC90701D1C043410800B506F000FA29
:101C50000022002300BD00B500290ADBDB4352420D
:101C600000D1013300F014F8C943404200D10131E2
:101C700000BDC943404200D10131DB43524200D193
:101C8000013300F005F8DB43524200D1013300BDBF
:101C9000002923D1002B18D1002A0CD0BC460D4FAF
:101CA00038667A6600210023FFE7FFE7FFE77A6FD7
:101CB000386F67467047002801D00748010000B51B
:101CC00006F0C6F90022002300BD02000B00002030
:101CD00000217047000000D0FFFFFFFF002B00D065
:101CE000BFE0130C28D1002AE7D080B4114F396629
:101CF0007A66FFE7FFE730B4040C7B6F396F1B0493
:101D000023433B667A66FFE7FFE7FFE7C04684B2FE
:101D10007B6F3D6F1B0423433B667A66FFE7FFE75B
:101D2000C04600232C042D0C7A6F386F00196941CE
:101D3000B0BC7047000000D0F0B594460025140EEA
:101D400001D112020835140F01D112010435940F8C
:101D500001D192000235D40F01D152000135D40BCC
:101D60000134254F7C66254C3C660E0C93B2FFE790
:101D7000FFE7FFE73C6F6643360C7703BE467343CD
:101D8000DF0B5B04C01AB941130C7343DB18C91A8B
:101D9000CE086643360CB64493B273431F0F1B0143
:101DA000C01AB941130C73431F0B1B05C01AB9416C
:101DB000860D8F023E436643360C092D24DB520A02
:101DC0007243801A7703460A6643360C16235B1B60
:101DD000DE40DF40BF1964466643821B704604350F
:101DE00006330100D940A840C01900D30131A242F6
:101DF00006D20023F0BD0000000000D0FFFFFFFF6F
:101E0000121B0130F3D3F1E709277F1BFE40644624
:101E1000A2B27243801A00D20139220C7243130C11
:101E20001204821A99410B007046043513370100E1
:101E3000F940A840801900D30131002B02D1A24201
:101E40000AD2F0BD013000D30131121BFAD2013B9E
:101E5000F8D1A24200D2F0BD013000D30131121BF3
:101E6000F7E7F0B51C0C00D080E00CB400251C0A8C
:101E700004D11B02160E3343120208351C0B04D189
:101E80001B01160F3343120104359C0B04D19B0038
:101E9000960F334392000235DC0B02D192185B415E
:101EA00001351C00971864410134464F7C66464C4E
:101EB0003C660E0CFFE7FFE7FFE7C0463C6F66435A
:101EC000360C7703BE4697B27743C01B00D2013968
:101ED000C01B00D201399FB27743C91BC91B170C25
:101EE00077437E04FF0B801BB941CE086643360C56
:101EF0000C2D33DBB644120B1F053A431B0B97B274
:101F00007743C01B00D201399FB27743C91B170C1E
:101F100077433E043F0C801BB941860D8F023E4340
:101F2000664329277F1BFE400C3D7746AF40BF1913
:101F300030BCA2B2ABB272437343801A9941220CF7
:101F40007243130C1204801A994102000B000137EE
:101F5000001BA941F9D2781E0021F0BD0C277F1B80
:101F6000FE4077467F0BAF40FF19E0E700245D1C81
:101F700007D0144F7D663966FFE7FFE7FFE7FFE70D
:101F80003C6F95B29EB265436643401BB141150C50
:101F90001E0C6543664336042F0C3E432D04401B44
:101FA000B141994204D202000B0020000021F0BD93
:101FB00001D19042F7D3801A994101349942F2D36A
:101FC000F6E70000000000D0FFFFFFFF484041405F
:101FD000484018B41B4B5B68FC46019308BD04DF06
:101FE0008F22001018B4174B1B68FC46019308BDE4
:101FF00000DF992200109446134A926F920809D28A
:10200000624618B40F4BDB68FC46019308BD0CDF39
:10201000512500100C4AF0B5146E556E576F166FAF
:102020006246FFF7EEFF084A146655665767166763
:10203000F0BD18B4034B9B68FC46019308BD08DF54
:10204000F5230010A8170020000000D0FFB5504075
:102050004240504059404B40594000E0FFB5154FB9
:102060004C00640D03D0BC4204D10C0314D80020F2
:10207000090D09055C00640D03D0BC4204D11C03AA
:102080000AD800221B0D1B0501264B4009D44B40EA
:1020900003D58B4200D18242FFBD9942FCD19042D0
:1020A000FFBD0B43DB1803431343F5D0C943491865
:1020B000FFBD0000FF07000000B5FFF7CFFF804124
:1020C00000BDC04600B5FFF7C9FF01D9002000BD23
:1020D000012000BD00B5FFF7B9FF01D9002000BD08
:1020E000012000BD00B5FFF7B1FF804100BD012018
:1020F00040054A00121804D85A00121801D80020CE
:1021000070470120704700000021002805D170476A
:10211000C1174840401AFAD0C90713B5064B1B68CF
:1021200098470CBC441CA2401005120B0349091B24
:1021300009051943114310BD002800201F040000A9
:1021400010B54C00620D8023D218DB00D21A5B055B
:102150007E2A10DD9E3A13DACC1709034908194389
:102160005242D140640001341532202A05DAD040B1
:102170000843604310BD002010BD0846604310BDF9
:10218000C80FC018013810BD18B4044B5B6AFC4678
:10219000019308BD24DF012700100000A8170020CC
:1021A00018B4044BDB6FFC46019308BD7CDF81272C
:1021B00000100000A8170020132370B51D78012D12
:1021C00019D014DD1F48FFF725FB06001E48FFF756
:1021D00021FB1E4C80223100200000F0E3FB022D89
:1021E0002DD01B48FFF70EFB1A4B186070BD1A4B21
:1021F000164CA364F5E7184B144C23606360A3608E
:10220000E36023616361A361E36123626362A362AC
:10221000E36223636363A363E36323646364A3648C
:10222000E36423656365A365E36523666366A3666C
:10223000E36623676367A367E367A364D1E7064B9D
:10224000A364CEE75344000053460000A8170020C3
:102250004C330000002800205D22001007B56046C6
:1022600001880A0A0230DF2AFAD1C9B2820804D3EF
:10227000028840880004104300E00068014A505082
:10228000039007BDA81700200FB403BC0CBCF0B529
:102290000124E407634000E0F0B50C0DCF0F661E8B
:1022A0003605891B640503D3C943404200D301317D
:1022B000640D03D0661CF60A07D0E41B00207F00E3
:1022C000791C89078912803C24031D0DDF0F6E1EC7
:1022D00036059B1B6D0503D3DB43524200D301330C
:1022E0006D0D03D06E1CF60A07D0ED1B00227F0097
:1022F0007B1C9B079B12803D2D032F1B661B58D414
:10230000A446202E46DA20371400BC401D00BD40F4
:10231000F24033412A4380185941CB0F05D0C943BD
:10232000C043002264425041514162464D0D28D1C4
:102330000D0D07D100281FD0241940414941013A11
:102340000D0DF9D0640006D3013000D30131002C0B
:1023500001D140084000013A0BD4941CE40A04D196
:1023600012051144DB071944F0BDD907204B19436E
:1023700000E0D9070020F0BD0029DDD1002CDBD121
:10238000F0BD0132C6074008CD0728434908002E9A
:10239000E1D0D9E73C2E29DA203E40371400BC407A
:1023A00000D00124F24014431A00BB401C43D31751
:1023B000ACE7AC46202F08DA20360400B4400D000C
:1023C000B540F84039412843A5E73C2F0CDA203FBF
:1023D00040360400B44000D00124F8400443080013
:1023E000B1400C43C117EAE710001900002494E73C
:1023F0000000F07FF0B50C0D661E3605891BE60A5D
:102400006405640D02D0651CED0A04D00020012192
:102410000905803C2403A4461C0D671E3F05DB1BF9
:10242000E70A6405640D02D0651CED0A04D00022A1
:1024300001231B05803C24037740644497B484B295
:1024400096B27443070C7E43150C6F4380B2684309
:10245000361802D3012000043F183004350C00194F
:102460007D41844688B29AB250430C0C62431F0CE3
:102470007C438EB27E43921902D301263604A419FE
:102480001604170C3618674101BC81B29AB2514349
:10249000040C62431B0C5C4380B25843121802D3F5
:1024A0000120000424181004130C401863412D1857
:1024B0005E410020474106BC88B293B258430C0CE1
:1024C0006343120C544389B251435B1802D3012178
:1024D0000904641819041A0C091862416D18564150
:1024E0000020474118BCF902720D1143F0026A0D39
:1024F0001043ED020A0D03D16D1940414941013BE2
:10250000124E9B1B7600B3420ED26D0007D30130F2
:10251000002671416646354301D1400840001B0545
:10252000C918E4072144F0BD0BDA013306D10130AC
:1025300004D101314F0D01D04908F2E7E107002035
:10254000F0BD013631050020EBE70000FF0300007D
:10255000F0B51C0D671E3F05DB1BE70A6405640D23
:1025600002D0661CF60A04D0002201231B05803C21
:102570002403D0252D060026F6432E661E096E661E
:10258000CE0FF619B44649004F0D02D07E1CF60A54
:1025900003D000200021403F3F033E1BB600B4445F
:1025A000013F7F05C91B49082E6F013676089C0242
:1025B000950D25437543ED137543AD1301356D102E
:1025C000F603761B0CB4CC02450D2C43A2B2B3B279
:1025D0005A43270C7B43350C6F43A4B26C431B1941
:1025E00002D3012424043F191C041D0CA4187D41AE
:1025F00024196D41009A91B2ACB26143170C7C432F
:102600002B0C5F4392B25A43A41802D30122120446
:10261000BF182204230C52187B41019C6C431B19E8
:10262000520ED9010A434401A01A81B2B2B25143F9
:1026300003145A43360C734387B27743D617D21923
:1026400000277E4136049B191704160C7F185E4143
:102650007316ED18F301002680337541A90F06D1DA
:102660006400690AE8055B0A184309D22FE00422D6
:10267000944480337541A90AA8059B0A184326D3C0
:10268000404149412404009A019B0D005543641BBD
:102690004343E41A95B286B27543170C7E43030C8C
:1026A0005F4392B25A43B61802D301221204BF18F4
:1026B0003204330C52197B4152429C41002C02D40B
:1026C0000022013051414008CA071043490802B0B6
:1026D0006246D7079210084BD218084B9A4203D291
:1026E00012058918C919F0BD0020002A01DC390043
:1026F000F0BD01331905F5E7FD030000FE070000FA
:10270000002200B5203200F004F8080000BD0000EF
:1027100000220B150AD410B5944600F05FF814148B
:10272000013400DA0021CB17144C2047002000218F
:1027300070476244343A0CD40C2A07DA0400914002
:10274000904052422032D440214310BDD843D94357
:1027500010BD203207D40C46944052422032114121
:10276000D040204310BD0800C917203203D4524284
:102770002032104110BD1800190010BD3327001081
:102780004A00520D144BD21A13DDFF2A1EDAD2056D
:10279000CB0FDB071A43C300400F0903490A084364
:1027A00010435B0001D301D0013070474308FBD2D6
:1027B000704702D0C80FC00770470A0312130132D6
:1027C000F8D1420F072AF5D1012200E0FF22C80FFD
:1027D00000028018C0057047800300000A0DCC0F6E
:1027E000531E1B05C91A520503D3C943404200D3E7
:1027F0000131520D03D0531CDB0A07D0121B0020FD
:102800006400611C89078912803A1203014BD21AB5
:1028100070470000FF03000051434343C9188C4632
:10282000110C83B24B4310B4040C614392B280B2DA
:10283000504362431C041B0C001910BC5941130483
:10284000120CC018514161447047000007B5484060
:102850004140484001E0C04607B54200120E03D097
:10286000FF2A03D1420218D8C00DC0054A00120E3B
:1028700003D0FF2A03D14A020FD8C90DC90501228E
:10288000414005D4414001D5814207BD884207BD82
:102890000143491801D0C043001807BD00B5FFF738
:1028A000DBFF804100BDC04600B5FFF7CFFF804190
:1028B00000BD0000034BDB6FFC4618477CDF592945
:1028C00000100000A8180020132310B512481C782F
:1028D000FEF7A0FF0100012C0AD003DD80220F4883
:1028E00000F060F80E48FEF78DFF0E4B186010BD2B
:1028F0000A4C5422200000F055F80B4B6365A36589
:10290000E36523666366A366E36623676367A3677D
:10291000E3672362E361E5E753460000A81800205F
:102920004C330000002800202D29001007B5604618
:1029300001880A0A0230DF2AFAD1C9B2820804D318
:10294000028840880004104300E00068014A5050AB
:10295000039007BDA8180020C30FDB0741000A0E33
:1029600007D0FF2A08D00909054A891819434007EA
:1029700070471900002070470249C918FAE70000A3
:10298000000000380000F07F01480421014B184787
:102990006010002025180010014B1B68184700002C
:1029A00060100020014B5B68184700006010002099
:1029B0007047C046F8B55746DE464E464546E0B538
:1029C00099460A9B07009A460D9B884693460B9CA6
:1029D0009B073BD10C9B9C423DD21E1B0B941500C8
:1029E0000C005E442A004B46013521002020B847E8
:1029F000B542F7D1A0460B9C002C20D04546361995
:102A00005346321B013C185D29004B46B847002C49
:102A1000F6D12B00350098460D9B9B070FD55B46E2
:102A2000EC1A0C9BA3420AD9464698462A004B460C
:102A3000310020200134B84701354445F6D3280041
:102A4000F0BCBB46B246A946A046F8BD160015002C
:102A5000002CD3D1E0E716001500002CCED1EEE714
:102A6000F0B54546DE4657464E46E0B585B09C4635
:102A700010AB1B78149F934698460F9C129E139D93
:102A8000BB074CD4002D42D1B44248D201233B4075
:102A900099460E9B013B9A46302304E0524601348E
:102AA0001355A64201D9202CF8D14B46002B00D15A
:102AB00083E00E9B013B99463023A54205D82EE0CA
:102AC0004A4601341355AC4229D0202CF8D1FB06DC
:102AD0000CD57B0554D4A64263D0A54261D0119B8E
:102AE000102B50D0022B57D0202C32D12023019311
:102AF0000E9B5A460093039763460295FFF75AFFD1
:102B000005B0F0BCBB46B246A946A046F0BD0123C5
:102B10003B40994601233B422AD1B442B9D3FB063C
:102B20001CD57B05DBD4002CD5D1119B102B5BD0A1
:102B3000119B022B6BD0302301240E9A1370434655
:102B4000002B10D17B073ED52B260E9A631C165501
:102B5000CDE72300013430260E9AD654202CC5D060
:102B60004346002BEED02D260E9A631C1655BEE769
:102B70004346002B2FD0013DB44200D289E798E7AD
:102B8000119B102BB2D1BB0637D5202CAED05823C9
:102B90000E9A13550134A7E7202CA7D02300013447
:102BA00007E0631E012CC0D0119A102A31D0022AEE
:102BB000D1D162260E9AD65496E7FB06CED57B0578
:102BC00000D488E78BE723003E0790D520260E9A95
:102BD000013316558BE70C233B405A1E9341ED1AE7
:102BE000B44200D255E764E7BB060ED478230E9AB0
:102BF0000224137030235370A1E7202C00D175E715
:102C000078230E9A135501346EE75823EFE76033AB
:102C1000EDE70E9AA61E91464E44BA0602D55822FA
:102C2000327098E77822327095E7C04610B50028D8
:102C300000D110BD01F046FDFBE7C0460B0010B50A
:102C4000002802D049681B68984710BDF0B5574668
:102C5000DE464E464546E0B595B083460F009246A7
:102C600098461E9A1F9B10001900209EFFF73FFAFE
:102C7000002800D0EAE11E981F990122C54B52425C
:102C8000FFF71AFA002800D014E11E981F990122BC
:102C9000C14B5242FFF726FA002800D0E9E01E9807
:102CA0001F990022BD4BFFF71DFA002800D0C8E095
:102CB0001E981F990022BA4BFFF7FEF9002800D09A
:102CC000BFE01E981F9900220023FFF7F5F90028A6
:102CD00000D0E4E000230B93229B5B0500D4062682
:102CE0000024302307E0172106AA01345218135597
:102CF000013E202C01D0092EF5D81E981F99FFF710
:102D00001FFAA84BF2009B181A685B68050008922E
:102D10000993FFF7FDF902000B001E981F99FFF7BA
:102D200058F9089A099BFFF784F906900791FFF775
:102D30002BFA8146FFF7E8F902000B000698079985
:102D4000FFF747F90022984B06900791FFF7CAF961
:102D5000002800D10DE101239C46E1444846FFF7DD
:102D6000D3F902000B0008980999FFF7ABF9002886
:102D700002D0002399460135002E00D1D9E00695F6
:102D80004D46B94614E006AA944617230A21634427
:102D9000280001341F19FEF7E1FE30313970280098
:102DA0000A21013EFEF7DAFE092D00D817E10500E1
:102DB000202CE8D14F46069D20240CAE06AA1723EE
:102DC0009446634499465B46B34606930FE04B46F0
:102DD00028000A210134E618FEF798FE3031280059
:102DE00031700A21FEF792FE051E00D1E4E0202C8E
:102DF000EDD1069B5E469B460323229A1340012B8E
:102E000018D1219B002B15D00B9B002B00D1FDE08E
:102E1000219B013B2193202B0CD93023219A07E0E1
:102E2000172006A9013409180B55944200D3CCE0B1
:102E3000202CF5D1229B01940393219B00960293B1
:102E400022E0229B52460493219B3900039358466B
:102E50001E9B1F9C029600930194434600F04AF982
:102E60000400200015B0F0BCBB46B246A946A046FF
:102E7000F0BD229B5B070FD403224C4B2299019299
:102E800003912199009302914346524639005846D6
:102E9000FFF790FD0400E4E70422454BEEE71E9A9D
:102EA0001F9B00200021FFF794F801231E901F9123
:102EB0000B9311E7229B54469B0711D1219B042BB6
:102EC0000ED9219B55469C465E46043C64442A002C
:102ED0004346013539002020B047A542F7D1B3461B
:102EE000344D26002B1F99465B46A3461C0032003A
:102EF000E87843463900013DA04701364D45F6D1FB
:102F000023005C469B46229B04349B07A9D553466D
:102F1000219AE31A9A42A4D95E461500220043463C
:102F200039002020B04753460134E31A9D42F5D8BA
:102F300097E72800FFF7ECF802000B001E981F9996
:102F4000FFF747F80022184B06900791FFF7B4F8F7
:102F50000CAE002800D031E7069807990022124BEA
:102F6000FFF7C0F8002800D028E7012301359D4372
:102F700024E70022069807990B4BFFF79DF80028DD
:102F800000D0F9E64B46002B5CD101239C46E1447E
:102F9000F2E6C046FFFFEFFFFFFFEF7F65CDCD41BB
:102FA00065CDCDC1E08600100000E03F3C840010FC
:102FB0003484001044840010069B5E469B46032325
:102FC000229A1340012B00D181E0202C00D131E75F
:102FD0000B9B002B27D02D23335501342AE74F4676
:102FE000069D202C00D1E7E63022331907E0172098
:102FF00006A9013409180A55202C00D1DCE6A342A9
:10300000F5D12E220CAE0134F254D7E60C23229ACD
:10301000134257D0219B013B2193A34200D9FCE6E8
:10302000202C00D106E7229B5B0703D52B233355C9
:103030000134FFE6229B1B0700D4FBE62023335517
:103040000134F7E6DB0700D496E69EE7229B55465F
:103050009B0711D1219B032B0ED9219B54469C46E3
:103060005E46033D6544220043460134390020207A
:10307000B047AC42F7D1B346B9465F461C4EEC1C94
:103080002A00B078434649460135B847013EAC4274
:10309000F6D1229BBB464F469B0700D4E1E6534640
:1030A000219AE31A9A4200D8DBE65E461500220018
:1030B000434639002020B04753460134E31AAB425F
:1030C000F5D3CEE6219BA34200D9A6E6B2E6219B2A
:1030D000002B00D179E70B9B002B97D0219B013B64
:1030E00021939C4200D298E6202C00D073E7A1E601
:1030F00040840010F0B5DE4657464E464546E0B5E2
:1031000099B081468B4692469846229A239B10009E
:103110001900FEF7ECFF002800D0CAE0229823999E
:103120000122824B5242FEF7DDFF002800D0C0E0B2
:103130002298239901227E4B5242FEF7BDFF0028C0
:1031400000D0B6E02298239900220023FEF7B4FFB6
:10315000002800D0C9E1229B239C08930994089879
:1031600009998023269ADB001A400D928022269C22
:103170001201144022000B94269C07000E001C42F2
:1031800000D0ADE00B00034300D0D5E0002A00D012
:103190000AE2220006332493022313400C930223F5
:1031A000134200D002E2259B042B00D20FE2043B25
:1031B0000B93002304250A930022229823990023CD
:1031C000FEF77AFF002800D003E25A4B269A1340FC
:1031D00004930B9B0393249B0293089B099C0093ED
:1031E00001945946434652464846FFF72FFD0200D8
:1031F0002020269B1F27034059424B415B42184029
:10320000531C0893594643464530C8470A9AD3177A
:10321000D4185C40D30F0A936B1E0B9308AB9C46EB
:103220000025674401E0202D0FD020000A21FEF781
:1032300095FC01357E193031317020000A21FEF7EE
:103240008DFC26000400092EEDD8052306930B9B68
:1032500059460593002304930A3303930A9B484677
:10326000029310AB0093089A43460195FFF7F8FBD1
:103270000C9B002B2DD05346C41A259BA34228D962
:103280004D465F4681461E00534639001A192020DC
:1032900043460134A847A642F6D8534648462599E6
:1032A000C21A01320023914200D386E1013018187E
:1032B0000FE0269B0493259B0393249B0293229B60
:1032C000239C009301944346524659464846FFF7D3
:1032D000BDFC19B0F0BCBB46B246A946A046F0BD45
:1032E00001432BD10B9B2200002B00D154E700237C
:1032F0000A93249B0A9A0024934200DD85E12298D8
:10330000239900220023FEF7D7FE002800D035E1E4
:10331000269B084A02941A408023DB00134304933F
:10332000259B0393089B099CCBE7C046FFFFEF7FDB
:10333000FFFFEFFFFFF7FFFF06232493B44B70005E
:103340009C46400D6044FEF7E3FEB24AB24BFEF7E6
:1033500070FEB24AB24BFEF745FE3603B14B360B58
:10336000334304000D00380019000022AE4BFEF775
:1033700030FEAE4AAE4BFEF75CFE02000B002000B2
:103380002900FEF72FFEFEF7DBFE0A90FEF7C0FED7
:10339000A84AA94B04000D00FEF74BFE0022A74BE4
:1033A000FEF720FEFEF7CCFEA54A0600A54B200046
:1033B0002900FEF73EFE040030000D000C96FEF7DB
:1033C000A7FEA14AA14BFEF734FE02000B0020002D
:1033D0002900FEF7FEFD02000B0006000F00FEF7BD
:1033E00028FE320004000D003B0030003900FEF7DB
:1033F000F9FD00220E900F91954B20002900FEF759
:10340000FAFD0022934BFEF7EDFD02000B002000B9
:103410002900FEF7F0FD00228F4BFEF7E3FD0200CE
:103420000B0020002900FEF7E6FD0D0080210400BE
:1034300032003B000020C905FEF7CBFD02000B0067
:1034400020002900FEF7CEFD02000B000E980F9918
:10345000FEF7D1FD0022734BFEF7C4FD7F4B0C9CA1
:103460009C46644400222305FEF7E3FD06000F009E
:1034700002000B0008980999FEF71EFE00280AD0EA
:103480000A9B3000013B39000A930022714BFEF782
:10349000B2FD06000F000A9A330063323900C62AD3
:1034A00012D802222698042510400B9A0C90002A6C
:1034B00025D1259B042B05D9002800D0A1E0259B10
:1034C000043B0B93042541E00222269810400B9AFE
:1034D0000C90002A12D1259B052B76D9002872D199
:1034E000259B0525053B0B9334E08022120694466C
:1034F000229B0893239B6344099330E605250B43E5
:1035000000D1F6E608980999554A564BFEF7E2FDB8
:10351000002808D0089809990022534BFEF7CCFDEB
:10352000002800D0E5E6249B002B1CD00D9B002B2F
:1035300019D0249B013B2493259BAB4204D90C9BBF
:10354000002B5AD002230C9300230B930A9B002BD1
:1035500000D131E60898099932003B00FEF74BFD97
:103560000890099128E6259BAB42EDD90C9B002BD6
:1035700043D000230B9302330C93E7E78020269B74
:103580003A4A00061A40802384460294089C099D0A
:103590002900DB0013430493259B6144220003931D
:1035A0000B00009201938EE60524A8E600230B93FE
:1035B0000A93023304250C93FEE553468C46013BE7
:1035C00063441B1A72E602230C930525C2E7042309
:1035D000EDE58020089E099F000639008446269A62
:1035E000224B6144134004930B9B32000393249BB2
:1035F00002930B0000920193F3E5259B5B1B0B9359
:10360000A4E7022304250C93A0E79C1A013C76E66C
:1036100001FCFFFFFB799F501344D33FB3C8608B7D
:10362000288AC63F0000F03F0000F83F61436F6307
:10363000A787D23F71A379094F930A400000E03F6A
:103640001655B5BBB16B0240EF39FAFE422EE63F8C
:1036500000002C400000244000001840FF03000040
:103660002D431CEBE2361A3F80842E41FFF7FFFF0B
:10367000F0B5DE4657464E464546E0B5A5B01E00BD
:103680002E9B92460C93CD4ACD4B80468B461A60BA
:10369000002900D1EAE1002330789946002800D1C2
:1036A000ECE1C84B4C460B93C74B454657460E932F
:1036B0000AE0631C984622003B005946A84744464E
:1036C0003078002800D187E001362528F1D1082381
:1036D0009A46043B9946023B9846013B00229C4691
:1036E0000D943078711C0300203BDBB2102B03D803
:1036F0000B9C9B00E3589F460300303B89460D9C82
:10370000092B3AD9002398462A2800D1C1E000238A
:103710009A462E284BD00300683BDBB2122B1ED8F2
:103720000E999B00CB589F4663460E001A43D8E77C
:1037300043460E001A43D4E74B460E001A43D0E727
:1037400010230E001A43CCE753460E001A43C8E775
:1037500080235B001A43FF3B9C467078E1444E4651
:1037600067284FD82428A4D90300253BDBB2422B7D
:103770009FD896499B00CB589F46002394461E0035
:1037800000E00131B3009B195B001E180878303E41
:103790000300303B092BF4D90123624689469C463D
:1037A0000023B0469A460E00E1442E28B3D13021C2
:1037B000802049428C46C000024370784B468444C6
:1037C0006146092900D86CE12A2800D17AE1012359
:1037D0009C464E46E1449EE7A146A846BA46CA45E5
:1037E00003D801235B425344994653464A465946FF
:1037F0000020C047200025B0F0BCBB46B246A94619
:10380000A046F0BD0300693BDBB20D930F2B00D93E
:103810004FE7012199408C466D49894661464B46E8
:1038200019400F91634649460B4200D028E10D9B99
:103830000A2B3AD0072B00D03BE70C9B190008C994
:103840008846002B00D14BE121200243914614A968
:103850008C461F220F2162448C4651460D950C91D7
:10386000A24615000F9902E020290CD013006446EF
:103870001C4020003730092C00D80738013168542B
:103880001A090F2BF0D80C9B54460D9D9A460F91A8
:1038900033E10C9B02CB8846002947DB0C930123C4
:1038A0009C4670784E46E14431E70C9B02CB149362
:1038B0005346002B00D138E19C4608780B000C9051
:1038C0008C44002801D100F098FC8946614694465A
:1038D00003E05A780133002A01D08B42F9D14946DE
:1038E00062465B1A0C900F93530500D520E102232A
:1038F000180010400D90134200D1CBE30D930B1B29
:10390000B1469A465E460C9822003B003100A8471B
:1039100053460134185D0028F6D1B3464E460D9B40
:10392000002B00D0C7E1149B0C93C9E60C93012334
:103930009C46283849420243884670784E46E14406
:10394000E5E670786C2800D17FE180235B001A43A4
:10395000FF3B9C46E14402E780239B001A4301237E
:103960009C467078E144FAE67078682800D173E1EB
:1039700080231A437F3B9C46E144F0E6672800D150
:1039800003E1472800D15AE1452800D15AE10492C9
:10399000072142460C9B0392073352468B43190082
:1039A00002920CC92800009201930C9122003B0066
:1039B0005946FFF79FFB040082E6C04671360010AF
:1039C000D42700204485001088850010D48500107D
:1039D00041900000462800D1DBE0049207214246D6
:1039E0000C9B0392073352468B43190002920CC979
:1039F0002800009201930C9122003B005946FFF7EA
:103A000025F904005CE6631C984622003B005946F9
:103A10002520A847444653E60C9B04330D93631CB2
:103A20009946920700D422E10C9B2200187859464F
:103A30003B00A84743464444012B00D885E23300AD
:103A4000B8462E005F4625004C4699462200434664
:103A5000013439002020B047AC42F7D12C00BB46DE
:103A6000350047464E460D9B0C9329E6DB4B3078DC
:103A7000984600239946002800D012E60024AEE6BE
:103A80006F2800D188E000D80BE31023782800D1FC
:103A9000CFE09A430A239C4600230F930A330D93E9
:103AA00080E05646B1008919490001330E18187894
:103AB000303E010030390929F4D9B2461E000133E5
:103AC000994628E60C9B023602CB8A46C9435046EB
:103AD000C917084082460C933078731C99461AE641
:103AE000102310009843113318438146802013009F
:103AF000C0000340024200D1A9E64B4606930823CA
:103B000005935346049310230393002302930F9BC2
:103B1000220001931CAB009359463B002800FEF79E
:103B20009FFF434604000C93CAE501235B42C3E6B2
:103B30000F9B534501D953460F93022318001040A1
:103B40000D90134200D1B7E10D93D1460B1B9A465D
:103B50003300A1442E0022004D460C98B9465F4622
:103B60009B4608E04B463900541CB0475346185D4D
:103B7000002877D022009542F4D15B46BB464F46E1
:103B8000A94635004C461E00C9E680231B011A4396
:103B9000FDE620231A4320E708239C4600230F93C9
:103BA00008330D9380231100DB0019401A4200D125
:103BB00016E10D239A431000802302009B001A4057
:103BC0001492184200D0C2E1802302005B001A4028
:103BD00091460C9A04320F92184200D0B7E2430685
:103BE00000D59FE1030600D419E30C9B1B880993C1
:103BF000002B00D0FCE110339843002900D1F7E1FD
:103C00000023994643460593534604930D9B069023
:103C100003930023D2E0582808D0622867D10223FA
:103C20009C4600230F9302330D93BBE720231A43D6
:103C3000103B9C4600230F9310330D93B2E7802373
:103C40001B011A4320231A43A1E6C0239B001A43F9
:103C5000F31C9946B07882E5C0231A43F31C9946B9
:103C6000B0787CE535005E46BB464F4657E6434696
:103C7000012B00D863E1631E43449A463300B946E2
:103C80002E005F4655469B46A24622004B46013415
:103C900039002020B047AC42F7D135005E46BB4624
:103CA0004F46A14654460C9B4A46187859463B005D
:103CB0004444A847D7E6A1460F9B984500D832E672
:103CC0004444E41A3300B8462E005F4625004C46B3
:103CD000994622004346013439002020B047AC42C7
:103CE000F7D12C00BB46350047464E461BE68023E5
:103CF0001000DB0018401A4200D10FE1112118001A
:103D00008A430D920D9A802311009B0019408C4626
:103D10001A4269D1802311005B00194089460C9931
:103D200004310F911A4200D0CAE113005B0600D59E
:103D3000F0E013001B0600D459E20C9B00229B5EAE
:103D4000D9175A184A4092B2D90F0C91002B00D1C2
:103D5000F9E1100014AA944642461F2314925246D9
:103D60006344A84616944D460400B946B2461F0067
:103D7000159201E0202D0FD020000A21FDF7EEFE64
:103D800001357E193031317020000A21FDF7E6FE41
:103D900026000400092EEDD8149B4F46A94645463F
:103DA0009846159B56469A46169C0D9B069343468D
:103DB0000593534604930A2303930C9B02934B46AB
:103DC00001931CAB2200009359463B002800FEF7EC
:103DD00047FE0F9B04000C9372E4C046B12900100B
:103DE0000C239A431000E7E607220C9B073393430A
:103DF000013294469C4462460C920CCBD90F0F9131
:103E00001100194300D191E0D9171391129151403B
:103E1000109113995940119110981199129A139B6E
:103E2000801A99411090119114AA00239446424699
:103E30009946149252461F336344A846B2461694DC
:103E40004E46109C119DB94615921F0001E0202E90
:103E500010D0200029000A220023FDF7BDFE013604
:103E600030322B00BA550D0022000400002BEED199
:103E7000092AECD8149B1094119545469846159B39
:103E80004F46B14656469A46169C0D9B06934346AE
:103E90000593534604930A2303930F9B02934B46C7
:103EA00001931CAB2200009359463B002800FEF70B
:103EB000D7FD0400FFF704FC0F9B984500D8C1E133
:103EC0008023DB000D9343460F9A1B199B1A9946DA
:103ED00033002E004D46B9465F469B460C912200AA
:103EE0004B46013439002020B047AC42F7D143465D
:103EF0000C9901330F930B7835000C935E46BB464B
:103F00004F46002B00D10EE50D9B002B00D1F6E4AF
:103F1000002319E60C9B1B781A0015E710239A431F
:103F20000D92EFE60C9B1B78099361E600239946FE
:103F30000028AAD1002200231092119374E70C9B51
:103F40002200187859463B00A8474C468BE50C9A4E
:103F5000FA3BFF3B07329A430133994691444B4663
:103F60000C931368526815921A4306D1103290438D
:103F700000220992002900D081E06122810600D54B
:103F80004122D2B20A9214AA91460A9A00210A3A10
:103F9000149242461792524618925A460991B346D5
:103FA0001F311E000F9B4944BA4619941A950024EC
:103FB000674698468946159D16901B920AE0303256
:103FC000D2B24B4601341A55A8454AD0202C4AD0CB
:103FD00006000D003A00002330002900FDF7FCFD2B
:103FE000D2B2092AEBD9149B9C466244D2B2E8E7CC
:103FF0006123820600D54123DBB20A3B0C93434682
:1040000014A91F228C46159353466244A046B2461B
:104010004C461797A9461700099D0D9E14901693BC
:1040200008E03033DBB201343B55B5420ED3202CCF
:104030000CD0050031002800FDF790FDCBB2092916
:10404000EFD90C9A94466344DBB2ECE7159B4D46DE
:10405000A14644469846169B564614989A46179F82
:10406000D0E5B742B2D9179B57469846189B5E4693
:104070009A461B9B09949B461698199C1A9D434689
:104080000593534604930D9B0690039300230293DC
:10409000099B05E70F9B984500D914E701330F935F
:1040A0002DE41023110099430D91692800D0BAE046
:1040B00080231000DB0018401A4200D122E61DE6E2
:1040C0000C9B1B68DA0F1100002B00D18CE0DA1773
:1040D0009818504014AA914642461F231492524603
:1040E0004B44A046A946169704006546B2461F00F9
:1040F0000C91159201E0202D0FD020000A21FDF730
:104100002DFD01357E193031317020000A21FDF777
:1041100025FD26000400092EEDD8149B4446984640
:104120000C9BAC461900159B56464D469A46169F69
:104130000D9B0291069343460593534604930A232D
:10414000039363463CE6002800D02EE602E60C9B73
:104150001B689946002B03D110339843002938D1AE
:104160006123820600D54123DBB20A3B0C93434610
:104170001693534614A91F228C4617932B006244B2
:10418000A0464D46B246189799461700149C0D9EBE
:10419000159008E03033DBB201343B55B5420ED305
:1041A000202C0CD0050031002800FDF7D7FCCBB245
:1041B0000929EFD90C9A94466344DBB2ECE7169BCD
:1041C000149444469846179B56464D469A46159871
:1041D000189F43460593534604930D9B0690039303
:1041E00000230293149BEBE50028A1D172E70C9BFE
:1041F0001B68D9175A184A40A6E580231000DB0037
:1042000018409C460F901A420FD002200300134022
:104210000F93104219D00023A1460F934CE50C9B3D
:104220001B680993E4E40A0034E4022318001040F8
:104230000D90134200D03EE54346002B00D042E6ED
:10424000FFF771FB01330F937FE463460D93F3E7B0
:1042500010B50C0084B00394012402A902900093CD
:10426000034813006242FFF703FA04B010BDC046D2
:104270003D2C001010B5094A0300146884B0002CCE
:1042800008D0012200910648524203A9A04701200C
:1042900004B010BD00F060FA0020F9E7D427002038
:1042A0002D2C001000BEFDE7094A0300106800280D
:1042B00005D00849C3188B4207D8136070470648D9
:1042C0000449C31810608B42F7D901204042F5E73A
:1042D000D0230020000004202C280020030010B56B
:1042E00008001100002B05D1044B1A685B6800F030
:1042F0004BF910BD01204042FBE7C046E8840010A6
:104300000300013B10B508001400012B06D801235F
:104310000022210000F0BAF8200010BD0120404228
:10432000FBE7C046012040427047C04601204042A2
:104330007047C04610B5FFF7B5FFC04670B5FDF732
:10434000C1FA074D074EB54209D20024013E761B43
:10435000B60808CD984723000134B342F9D170BDA7
:104360001C81001028810010030010B50800110006
:104370001B68984710BDC046F0B5C64600B5437DE2
:1043800007000C001600002B46D0002A17DD0B7822
:104390000A2B24D000239846012E13D00125290092
:1043A000635C01350A2B26D0B542F8D1464509DCBD
:1043B000A419013C23780D3B5A4253413B7580BC04
:1043C000B846F0BD4346E018A419F11A013C3B6819
:1043D000984723780D3B5A4253413B75EFE7037DE5
:1043E000002BD7D102210F483B689847012EDFD020
:1043F00001239846D2E7631E5B5C0D2BD4D0884521
:1044000004DA4346C91AE0183B6898470221054878
:104410003B68A8469847C7E7036811002000984703
:10442000CDE7C04630870010F0B5C6460B680600E1
:104430000C0000B5802B06D05A1C2260E4182671AF
:1044400080BCB846F0BD0F4B1D68002D16D00B1D6B
:1044500098460D4F02E02D69002D0FD02B68002BE0
:10446000F9D03B68002B01D0AB42F4D12800414683
:104470002268FFF781FF2D69002DEFD10122002373
:10448000DBE7C046C4230020CC230020F0B545461E
:10449000DE464E465746E0B583B091461C00804646
:1044A0000D00FCF7C5FF0023304A12184B41002BCA
:1044B00002DA01222E4B52422E4908008A4603F0AE
:1044C000E7FD07006B1C03D1404602F0A9FD050083
:1044D000002C27D0284E294B1C68002C18D04B46A6
:1044E000002B21D1264B994602E02469002C0FD0E5
:1044F0002368002BF9D04B461B68002B01D09C424F
:10450000F3D120002A004146B0472469002CEFD1A6
:10451000002F26D1280003B0F0BCBB46B246A94606
:10452000A046F0BD174ED6E7154B99460A239B4689
:1045300002E02469002CEBD02368002BF9D04B4615
:104540001B68002B01D0A342F3D12A004146200072
:10455000B0476B465A462000DA71D91D0122B04798
:10456000E7E7504603F064FDD4E7C04640420F0041
:10457000FFFFFF7F1816002079430010C42300209E
:10458000CC23002069430010F8B557464E464546F7
:10459000DE4698461A4BE0B59B461A4B07000E00C4
:1045A00091469A46184D5B461C68002C03D115E0D5
:1045B0002469002C12D02B68002B01D0A342F7D124
:1045C000A368002BF4D03100380098470028EFDDB5
:1045D000F0BCBB46B246A946A046F8BD53465B6A4E
:1045E000984508D85246926A4A4502D30220404272
:1045F000EEE79845FAD101200021FCF723FFD2E72E
:10460000C423002000400540CC2300200A4A136840
:10461000002B05D10CE01A001B691032002B07D0CB
:104620008342F8D1002902D11869106019617047DE
:104630000029FCD01060FAE7C423002010B500F078
:1046400031FB10BDF0B54746CE461A4B80B51A680F
:104650005B689146984683B0174F184D01AE3C6891
:10466000002C03D115E02469002C12D02B68002BFC
:1046700001D09C42F7D1A368002BF4D00121300077
:1046800098470028EFDD307803B0C0BCB946B0468B
:10469000F0BD0B4B5A6A904507D89B6A4B4502D335
:1046A00002204042F0E79045FAD101200021FCF7BA
:1046B000C9FED4E7E8840010C4230020CC230020E6
:1046C00000400540F0B5CE46474680B583B06B4606
:1046D0000600DD1D2870FCF7ABFE0023194A1218F6
:1046E0004B41002B02DA0122174B524217490800B6
:1046F000884603F0CDFC164B81461C68002C14D074
:10470000144F02E02469002C0FD02368002BF9D04D
:104710003B68002B01D09C42F4D1200001222900EB
:10472000FFF72AFE2469002CEFD14B46002B05D160
:10473000300003B0C0BCB946B046F0BD404603F0FF
:1047400077FCF5E740420F00FFFFFF7F18160020BF
:10475000C4230020CC23002070B5040002F060FCCC
:1047600001230100050001222000FFF78FFE084B06
:104770001C68002C06D06368002B05D0984724697C
:10478000002CF8D1280070BD2469002CF3D1F9E782
:10479000C4230020F0B5CE46474680B5A3B0040040
:1047A0000D00FCF745FE0023274A12184B41002B51
:1047B00002DA0122254B5242254E300003F068FCFC
:1047C00000232200019307002B00224801A9FFF7D4
:1047D0003FFD214B804699461C68019B002B1AD057
:1047E000002C2FD01D4D02E02469002C0FD023682F
:1047F000002BF9D02B68002B01D0A342F4D120006C
:10480000019A02A9FFF7B8FD2469002CEFD14B46AD
:104810001C6800230193002C06D06368002B0BD08A
:1048200098472469002CF8D1002F07D1404623B0C7
:10483000C0BCB946B046F0BD2469ECE7300003F0D7
:10484000F7FBF3E70194EFE740420F00FFFFFF7F24
:104850001816002029440010C4230020CC23002077
:104860000FB400B583B004A901C90191FFF792FF0D
:1048700003B008BC04B018477047C0460022014B83
:104880001A707047262800204B790020FF2B0BD18F
:104890008B79002B08D1CB79012B05D1082A03D9BC
:1048A000024B8A7809301A707047C04626280020CB
:1048B0000120704710B5012913D11249537910799D
:1048C00009781B0203430020994200D010BD5378A1
:1048D000012B08D0022BF9D1642200210020FCF723
:1048E0003BFF0120F2E7D37891781B021943480A75
:1048F000DB0501D4012040427F238A05D20F1940F5
:10490000FCF7B2FF2628002000487047FC87001003
:1049100070B5050014000120012909D15378002049
:10492000012B05D1637912791B021343072B00D0A9
:1049300070BD21002800024A9F3301F055FAF7E7C5
:10494000548700100123037000487047348700101B
:104950004B780A781B0213438A7810B512041A4365
:10496000CB781B0613439622D200934200D010BD91
:104970000022012011004042FCF776FF024B186034
:10498000024B19607047C046642300206823002052
:1049900010B5024B1878FBF72BFF10BD272800201D
:1049A000154B70B51A68002A22D0EFF3108172B649
:1049B00010680028FCD0BFF35F8F00200F4A5960B9
:1049C00010701B68BFF35F8F186081F3108800249C
:1049D00000250B4E3078FBF7FFFE002804D10024A1
:1049E00000252900200070BD3078FBF701FFF8E7B3
:1049F000FA240025A400ECE7E02700202828002066
:104A00002728002070B5040000200E0001F00AFBEA
:104A1000002834D0002001F01BFB00282FD0FCF729
:104A200007FD0023174A12184B41002B16DB164DC9
:104A3000280003F02DFB002821D0002001F0F2FA1D
:104A400000280FD101200021404200F001FD032485
:104A50006442280003F0ECFA200070BD01220B4BE9
:104A60005242E4E7002001F0F3FA0028EAD02100E6
:104A70003200002001F0F6FA041EEAD1E7E7032431
:104A80006442E9E740420F0008280020FFFFFF7F53
:104A900010B5FCF7CDFC00230D4A12184B41002B3A
:104AA00002DA01220B4B52420B4C200003F0F0FAC9
:104AB00000280CD001200021404200F0C9FC002059
:104AC00001F014FB0028F5D1200003F0B1FA10BD6D
:104AD00040420F00FFFFFF7F08280020F8B5DE46A8
:104AE000574680B505000C00FCF7A2FC0023364AAF
:104AF00012184B41002B02DA0122344B5242344946
:104B000008008A4603F0C4FA002803D1C0BCBB46A3
:104B1000B246F8BD002001F085FA00284AD00026F0
:104B2000002C43DD2B4B9B4614E0A919002001F01B
:104B300017FB070001200021404200F089FC002003
:104B400001F0D4FAFCF774FC224BF6191860596096
:104B5000B4422BDD002001F023FBA71B0200B8426A
:104B600000DD3A00002AE0D101200021404200F09F
:104B70006FFC002001F0BAFA002001F053FA00287F
:104B800014D0002001F00CFB0028E1D1FCF750FC10
:104B90005B460F001A685B68002184460E481218B5
:104BA0004B419F4202D8D3D19445D1D9504603F00E
:104BB0003FFAABE700200021064B186059605046D1
:104BC00003F036FAA2E7C04640420F00FFFFFF7F26
:104BD00008280020A017002020A1070030B52A4C8B
:104BE00085B00021200003F043FA00281CD1274B98
:104BF0001A68002A16D0EFF3108172B610680028E8
:104C0000FCD0BFF35F8F01242148596002781B68F4
:104C1000D2B20470BFF35F8F0020186081F3108858
:104C2000002A17D005B030BD01200021404200F01D
:104C30000FFC002001F00CFA0500200003F0F8F949
:104C4000002DEFD0134B1B68002BEBD0124A1068DD
:104C50009847E7E7FCF7D6F90400FCF7E9FBFA22EE
:104C60000023920012184B41002B02DA01220B4B59
:104C70005242012102910021019109492000009135
:104C8000FCF7C4F9CEE7C04608280020E027002042
:104C9000282800206423002068230020FFFFFF7FD6
:104CA000A1490010D02310B51B0684B01C68FCF786
:104CB000A9F9FCF7A5FAA04202D0002004B010BD6B
:104CC000294B002100201B7801F05EFD2748036876
:104CD000002B45D00120FBF723FFFF23244C25495F
:104CE00020701840FBF79EFD20780121FBF762FD44
:104CF0000520FBF785FD002824D1082200211E484D
:104D0000FDF74AFEFCF77EF90400FCF791FBFA225E
:104D10000023920012184B41002B02DA0122174B9C
:104D20005242012102910021019115492000009178
:104D3000FCF76CF90028C0DB12480121FFF766FC84
:104D40000120BBE70120FBF703FD0B4B010018001E
:104D5000FBF748FF002205200B49FBF78DFDEBE731
:104D6000FBF724FFB6E7C046B089001008280020F2
:104D700027280020DD4B0010E0270020FFFFFF7FE9
:104D8000A1490010701000209149001000487047A0
:104D900098880010004870474488001010B504003F
:104DA00017480378002B20D0002C06D1154B16484D
:104DB0004380063BFF3B038010BD052C1DD8134BE1
:104DC000A400E05812490123013804E001330A80AD
:104DD0000231142B0DD0C25C002AF7D1C022DBB205
:104DE0005B00920008481343E5E7112100F01AF830
:104DF000DAE7CA2304489B00DDE70020DCE7C04671
:104E000010280020090400009C2300202C8800109A
:104E10009E23002010B5024800F0D8F810BDC0460F
:104E2000F827002030B54B1E012900D1A7E0664AC3
:104E300011780D092C0030349F2900D9A2E00470AC
:104E4000012B00D1BEE00F21147821400C0030343A
:104E5000092900D998E04470022B00D1B2E05478BF
:104E60002509290030319F2C00D990E08170032B57
:104E700000D1A7E00F2121400C003034092900D9CE
:104E800087E0C470042B00D19CE0947825092900A8
:104E900030319F2C00D97FE00171052B00D191E0CA
:104EA0000F2121400C003034092900D976E04471EB
:104EB000062B00D186E0D4782509290030319F2CBB
:104EC00000D96EE08171072B00D17BE00F212140DA
:104ED0000C003034092966D8C471082B00D171E068
:104EE00014792509290030319F2C5FD80172092BD4
:104EF00068D00F2121400C003034092958D8447261
:104F00000A2B5FD054792509290030319F2C52D8C3
:104F100081720B2B56D00F2121400C00303409290F
:104F20004BD8C4720C2B4DD094792509290030310F
:104F30009F2C00D9073101730D2B43D00F21214045
:104F40000C003034092901D937310C0044730E2B81
:104F500038D0D1790C09220030329F2900D907328C
:104F600082730F2B2ED00F220A4011003731092AED
:104F700001D830321100C173102B23D01030002320
:104F8000037030BD07345AE737310C0063E707314F
:104F90006CE737310C0074E707317DE737310C00DF
:104FA00085E707318EE737310C0095E707319DE73C
:104FB00037310C00A3E70731AAE737310C00C47280
:104FC0000C2BB1D1C018DAE7F827002010B588B053
:104FD00004000D2200216846FDF7DEFC0D220021B1
:104FE00004A8FDF7D9FC4B236A466846137004A950
:104FF0000D2203F015F81521082220006944FDF761
:10500000D1FC08B010BDC046F8B500F047F90C233C
:10501000194DFF22AB6705201849FBF72DFC184CF2
:10502000402200212000FDF7B7FC40270023012685
:105030002121144A66702783A260136063545F3194
:10504000618445396354104A10496360E2602787E0
:10505000A1620B606362E26202F0F2FF80239B05B3
:105060002E64EB6490230A4A0120EA508022094B07
:105070005202DA64F8BDC046000011504505002018
:10508000D4230020840010500001105080001050E4
:1050900010D001000020115010B501210520FBF7B0
:1050A00089FB10BD10B500220021024800F016F95E
:1050B00010BDC046F4230020044B1970002904D011
:1050C00080219023024A8902D15070472228002073
:1050D000002011500B785B0602D14B78052B00D0D5
:1050E00070478A78014B1A60FAE7C04600001150F9
:1050F000F0B5C646C87800B58007830F1800012BAD
:1051000060D08F780A794B797F213940FC091B02E6
:105110004E001343334D32195201AA1897700127DC
:105120006740577000275B055B0DD7701383D076FF
:10513000B846CA00012C32D02B4FBC468F016244C6
:10514000BC46AC446746BA6047461760002932D077
:10515000264AC90090466246414451603F223F338F
:105160009343022837D0224937190A687F01D318A0
:105170000B602049EF19FA608B422ED83619760160
:10518000AD19EB7E1C499B064A4013438022120650
:1051900013436A681360012080BCB846F0BD174F06
:1051A000BC468F016244BC46AC446746BA6247467F
:1051B0001760002908D1002364012C196360104B8B
:1051C000E360E8E70020E7E70B4AC9009046624643
:1051D00041445162C2E75B00C5E7FCF76DFBFA682A
:1051E000CCE7C046D42300208400105004001050A7
:1051F000DC270020FF0F10500000105080001050DE
:105200000001105010B502F01BFF10BD10B57F203B
:105210000C0020404000E409110000191A00034B63
:105220004001C01800F05AF8012010BDD42300201E
:105230007F23180000B5084083B00B4204D14B42D5
:105240004B41084A013393668022C9094000064B4E
:10525000401840010021C018120102F031FF03B0D4
:1052600000BDC04600201150D42300207F2213002F
:1052700010B50B400A4200D110BDC9095B005B1894
:1052800004485B01C018002300220349C37002F0E8
:1052900017FFF1E7D4230020FFF7FFFF80220A4B1E
:1052A000520410B51A60094B09491A6010000B68C6
:1052B0009843FBD18022002152010648FDF76CFB88
:1052C0000922054B5A6710BD00E0004000F0004085
:1052D00008C000400000105000001150002310B51D
:1052E000C3820133828283760161040002F0E0FE12
:1052F000002804D080219023074A8902D150200041
:1053000002F0E6FE002802D00123237710BD200022
:1053100002F0C6FEFAE7C046002011507047C046B2
:105320007047C04600207047002070477047C04655
:105330007047C0467047C0467047C046024B587819
:10534000431E9841C0B270477C1E0020024B187863
:105350004007C00F7047C0467C1E0020F0B5D646FF
:105360004F464646C0B52F4B07009A461B780E00A5
:10537000FF2B50D1002941D0002154222A48FDF7AB
:105380000BFB0022294C2A4B20001A70FBF70EFC65
:10539000284B1C60284C2000143CFBF715FC200017
:1053A00001F0FAFD254B264D1C60264B002B04D046
:1053B0002800FFF7C7FA244B1860244900248946C7
:1053C0002149002388462A7810E043461B68620181
:1053D0009B18002B12D05B68002B0FD098472A78BF
:1053E0000134E4B2511C2300A14209DBA242ECD8F3
:1053F0009B1A5B014B445B68002BEFD100200BE054
:105400005346310038001F70FFF7FEFD0028F5D02D
:105410003800FFF741FE0120E0BCBA46B146A8467D
:10542000F0BDC046A41000207C1E0020741E002089
:1054300023280020D01E00209C100020D41E002015
:105440002128002045490010CC1C00205489001060
:10545000F0B5DE4657464E464546E0B5C84B91B0DE
:1054600002931B78FF2B00D13EE1C64BC64E9B46F4
:105470005F46C64B0DAC0193C54B009335686A6916
:10548000EFF3108172B61368002BFCD0BFF35F8F6F
:10549000A9612800210001F0AFFB6A69AB69BFF385
:1054A0005F8F0021116083F31088002800D11BE179
:1054B0006378082BE2D89B00FB589F466368002B5B
:1054C000DCD0A0689847D9E77F222179AF4D0A4008
:1054D0005300EB189846C8098044404601233030F9
:1054E00005799D430571057903339D430571002AB4
:1054F00000D100E14346A74A1B7D1278934200D3B6
:10550000EFE0A54A5B011568ED18002D00D1EBE036
:10551000A36862792078AD69A847AFE79F4A1378FE
:10552000002B00D1E0E01378013BDBB2137013785D
:10553000002BA3D10122954D01212B780420134388
:105540002B703423EA5C8A43EA54EA5C8243EA54CF
:105550000133EA5C8A43EA54EA5C8243EA542378E2
:1055600000209B4600F09EFC602223791A40602AAE
:1055700000D1EFE0402A00D1F5E0DB06DB0E012B85
:1055800000D113E1022B00D1C7E0002B00D0E1E0F5
:10559000202A00D11CE2002A00D0DBE06379092B2D
:1055A00000D9D7E07E4A9B00D3589F46774D2B7891
:1055B000DB0700D462E7FFF7BFFE5FE7019BDB7804
:1055C000DB0700D45AE76068FFF7AAFE56E76F4D85
:1055D0002B78DB0700D451E728780007C00FFFF7CE
:1055E000A9FE4BE723786A4999468B46694B6A497D
:1055F00098468A4639001A7847460023B046002567
:105600004E46894610E053461B686A019B18002BE2
:1056100000D176E0DB68300098473A780135EDB28A
:10562000511C2B008D4244DC9542ECD39B1A5B014C
:105630005B44EFE7237858499946564B8A4698468B
:105640003100BB464E461A7800250023474689465E
:105650000FE053461B686A019B18002B55D0DB688E
:10566000300098473A780135EDB2511C2B008D423D
:1056700007DC9542EDD39B1A009A5B019446634484
:10568000EDE7019D542200212800FDF785F9102245
:10569000FF214448FDF780F928002022FF21143023
:1056A0004E465F46FDF778F900F0F2FBFFF740FE4B
:1056B000E4E6364D542200212800FDF76DF9102252
:1056C000FF21281DFDF768F928002022FF21143052
:1056D00046464F46FDF760F900F0DAFB2379AB70E0
:1056E000CCE6501C984213DA11B0F0BCBB46B2466F
:1056F000A946A046F0BDA3686279207800F0E6FBD9
:10570000BCE646464F46214DE6E74E465F46CBE7B0
:105710001F4D9B1A5B015D19FAE67023217A0B423B
:1057200018D1C80982460F330B405B0098461948D0
:10573000EB1853441B7D00789946834266D2164885
:105740005B01006881469944002A00D15FE14B4625
:10575000002B68D120780021FFF76AFD8021207896
:10576000FFF766FD8AE6104800F09CFB01215846D1
:105770000EAAFFF7CDF8002800D07FE6EAE7C04682
:10578000A4100020AC880010D41E00207C1E002035
:105790005489001021280020CC1C00202328002040
:1057A000D0880010801E002011490010237A0F2B92
:1057B000D0D8CF4AEB181B791578AB423ED3691C81
:1057C0009942C7DB5D1BCB4B6D01ED18686900F09A
:1057D00069FB012158466B690EAA9847002800D042
:1057E0004CE66022150023791D401A42B2D163793C
:1057F0000A3B012BAED800F055FB63790A2B00D190
:1058000099E158460EA900F0D9FA37E6431C4B45FA
:1058100000DAF7E04B461B1A5B019946B548814414
:10582000002A00D1F3E04B46586900F03BFB4B46A1
:10583000012158465B690EAA98479CE7AE4A5B0176
:105840001568ED18002DC1D184E7A37999466B78CE
:105850009945D6D06B78002B00D033E14B466B7066
:10586000002B00D12BE148460138C0B2FFF792FA75
:10587000002800D17EE143780793022B00D079E124
:105880000122C179B1468B11491113400A403021E0
:1058900012015B0113432A78A8468A4313432B70F5
:1058A00009239A4682445646BA46C37882781B0238
:1058B0001343C31805938E4B04938E4B08938E4B62
:1058C00009938E4B0A93059BB34200D855E1737838
:1058D00001220B2B03D13378F278F6187378042B5E
:1058E00000D044E1059B00279B1B9BB20693049BC1
:1058F0000B921D78002303931BE0099A7B01156826
:10590000ED18002D00D132E1310058462B69069A7E
:1059100098478446082803D9069A824200D313E1A7
:10592000049B01371D78FFB26B1C03979F4200DD7B
:105930001DE1BD42E1D8039B5D1B089B6D019C46A8
:105940006544E1E76B780CAA0232137058460123D4
:105950000EA900F049FA91E5E3881A0AD8B20F2A95
:1059600000D9F7E666499300CB589F460EA800F091
:105970009FFA5846A179FFF795FB02222B78134333
:105980002B707BE5E388012B00D0E3E608222B781F
:10599000584693430EA92B7000F010FA6EE50220D2
:1059A00029780CAB9A1C8B068908DB0F01400B434E
:1059B0001380584602230EA900F016FA5EE5E3882C
:1059C000012B00D0C6E608222B7813432B7018E772
:1059D000237A0F2B00D9BDE6EB181D79444B1B78B9
:1059E0009D4228D2444B6D011B685D19002D00D1EA
:1059F000B0E6686900F056FA012158466B690EAAB4
:105A00009847B8E6002A00D0A4E6002399466279B8
:105A10000220130003928343012B15D0002A00D0EB
:105A200098E62B004344534430331B790CAA9B0760
:105A3000DB0F0232BCE75A1CAA4200DA8AE6ED1AF2
:105A40002C4B6D01ED18D4E7E388002B12D1029B9B
:105A50001878039B012B23D0FFF7EAFB4346022172
:105A6000EB18534430331A790A4301211A711A7919
:105A70000A431A714B46002B00D1FFE4586900F02D
:105A800011FA4B4601215B690EAA5846984700203F
:105A900000F008FA3523EB5CDB0700D5EEE4B0E656
:105AA000FFF7E4FB43460221EB18534430331A79E5
:105AB0008A431A711A7903998A431A71DAE7FFF750
:105AC00037FC9EE600215846FFF7F6FA5846FFF7E6
:105AD00099FBAB78074903930491054B0649984617
:105AE0001A780591002329001D008A461BE0C04654
:105AF0002128002054890010CC1C0020901E00207A
:105B0000F8880010059B6A011B689B18002B4DD07C
:105B1000DB685846984743461A780135EDB2511C68
:105B20002B008D422EDC9542ECD39B1A049A5B012C
:105B300094466344ECE70CAB9A1C584601230EA92B
:105B4000157000F051F999E40B9A012A4FD0002A00
:105B50003CD00023B07804E00133DBB20F719342F4
:105B600034D2C118C9B241440D79FF2DF4D04E464C
:105B70004546574600236B70ECE54E465746FFF707
:105B8000D5FB3EE65546542200212800FCF704FFD1
:105B90001022FF21281DFCF7FFFE28002022FF21F4
:105BA0001430FCF7F9FE039BAB7057E65546FAE755
:105BB000FEF7AAFE021E00D1CCE5D37891781B0235
:105BC0000B4358460EA900F00FF9D4E565463B009B
:105BD0002A0031000A9800F07FFEAC46049B039A2D
:105BE0001B7866440133934200DB6CE6BFE7174B3A
:105BF00029699942ADD1079AABE7FFF793FB021EE3
:105C000000D1A7E5584613780EA900F0EDF8B2E5EB
:105C10002189FFF7C3F8021EF4D19BE5022A0FD0B9
:105C2000FFF782FB021EC8D194E5FFF7AFF8021E12
:105C300000D18FE5122358460EA900F0D5F89AE559
:105C4000FFF7A8F8021EB8D184E5C046A162001093
:105C5000F8B557464E46DE4645460C00E0B5160000
:105C60001F00002A3CD0702398461E4B00259B46FF
:105C70001D4B9A461AE05B461B7820009946534616
:105C8000997800F0EBFD00281CD021004846FFF772
:105C90002FFA002816D0A378DA09012A19D00A9A17
:105CA000013513702378E418B54219DA6378052BAF
:105CB00008D1E3789B079B0FBB4203D14246A378F0
:105CC0001A42D8D00020F0BCBB46B246A946A04636
:105CD000F8BD0B9A013513702378E418B542E5DB63
:105CE0000120F0E7A41000207C1E0020702270B577
:105CF0008B780C001A4201D0002070BD064B2000AA
:105D00001D78064B997800F0A9FD0028F4D02100F9
:105D10002800FFF7EDF9F0E7A41000207C1E00201A
:105D20000B007F2010B51840DB0934334000044AD3
:105D3000C018044B1168C01800F04CFD10BDC046DF
:105D4000D01E00207C1E00200B007F2010B51840C4
:105D5000DB0934334000044AC018044B1168C018F2
:105D600000F060FD10BDC046D01E00207C1E00204B
:105D700070B57F240F480C4064000419CD096419E4
:105D800030342079C00701D5002070BD0126257967
:105D90000948354300782571FFF738FA0028F4D117
:105DA000012223799343237123790332934323718F
:105DB000EAE7C0467C1E0020A410002070B5094C04
:105DC0000600082220000D00FCF7ECFD00238021D6
:105DD000E360A3602B783000994300220023FFF793
:105DE000C7FF70BD5C1E0020F8B5CE464746904602
:105DF000254E80B58146082230000D001F00FCF7BB
:105E0000D1FD4346B3600023F381EC79AB792402E2
:105E10001C43231CBC4200D93B1C9FB2B381002C05
:105E20000DD0002F17D04246002A2BD0402F1BD870
:105E30009FB233787F2B1CD80021144A0FE08021B9
:105E40002B780022994348460023FFF791FFC0BCFE
:105E5000B946B046F8BD7F230022317899433B0014
:105E60004846FFF785FFF2E740239FB233787F2B48
:105E7000E2D9064C3A0041462000FCF793FD802110
:105E80002200ECE70020E2E75C1E00201C1E002040
:105E900010B5142200210248FCF77EFD10BDC0465B
:105EA0005C1E0020014B18617047C0465C1E00203C
:105EB00010B5054C010008222000FCF773FD0023FB
:105EC000A360E36010BDC0465C1E002070B5384C76
:105ED0001D0023780600DA09C9098A4210D0002083
:105EE000002D00D070BD21003000FFF7F3F82369CA
:105EF000002B03D022000321300098470120F1E756
:105F00007F2B06D8A068002834D02A002949FCF746
:105F100049FDE289A1685219E38892B24919E281E8
:105F2000A160934214D03F2D12D9A389981A051C61
:105F300080B240282AD82078ADB27F2828D8002106
:105F40009A4232D01B4A2B003000FFF711FFC9E7FD
:105F50002369002B05D02200022130009847002839
:105F60000AD0802123780022994330000023FFF7D4
:105F7000FFFEB7E70020B5E700213000FFF758F932
:105F800030008021FFF754F90120ABE74025D2E72C
:105F90009A4207D0074C2A002000FCF703FD80211D
:105FA0002200D0E780210022CDE70022CBE7C046C7
:105FB0005C1E00201C1E002070B50400FFF7BEF917
:105FC000002800D170BDFFF7C1F90028FAD1C8231D
:105FD0006343124DEE18F1780029F3D010335D19A8
:105FE000280000F0F3FD3F28ECD90020F178FFF7FE
:105FF00097FE0028E6D0280000F0E8FDF1783F2861
:1060000007D9074BE201D21800204023FFF7B0FE6A
:10601000D8E70020FFF798FED4E7C046541D0020C3
:10602000D01C002010B50400FFF788F9002801D12A
:10603000002010BDFFF78AF90028F9D1C822624379
:10604000024B01309B181B791840F2E7541D0020C9
:10605000C82310B543430248181800F099FD10BD3D
:10606000641D0020F8B5C824802344431C4F10341D
:1060700005003C195B029A4200D31A4A200092B2F2
:1060800000F008FE0600FFF759F9002801D13000A2
:10609000F8BDFFF75BF90028F9D1C8236B43FF185F
:1060A000FB78002BF3D0200000F090FD3F28EED9C4
:1060B0000020F978FFF734FE0028E8D0200000F037
:1060C00085FDF9783F2807D9074BEA01D21800204F
:1060D0004023FFF74DFEDAE70020FFF735FED6E755
:1060E000541D0020FFFF0000D01C0020F8B5040064
:1060F000FFF724F9002801D10020F8BDFFF726F9A9
:106100000028F9D1C82565432E00134F2436F6190F
:10611000300000F03DFD0028EED07F190020B97856
:10612000FFF7FEFD0028E7D00C4DE40165192900BA
:106130004022300000F0AEFDB978041E08D0030004
:106140002A000020FFF714FE0028D5D02000D4E755
:106150000020FFF7F9FDCFE7541D0020101D00209F
:1061600070B5C82444430C4B0500E41880235B023F
:106170009A4200D3094A200092B200F051FE060074
:10618000200000F005FD3F2801D8300070BD280038
:10619000FFF7ACFFF9E7C046781D0020FFFF0000C5
:1061A000C82310B543430248181800F00FFD10BD76
:1061B000781D0020F0B50025184C83B0C8220021BE
:1061C0002000FCF7E9FB164B21001D70FF236371D3
:1061D000E1235B02A360200008234022A37338312F
:1061E0000095073B103000F09DFC270001232100A3
:1061F00020002600402278310093B837243000F088
:1062000091FCC0363800FAF7D1FC3000FAF7CEFC2A
:10621000E56127622663656303B0F0BD541D00206D
:10622000501D00200A4A116B136A00290CD0002B64
:1062300007D00023D361536313630023136201204B
:10624000704753631363FAE7002BF8D0D161F4E78A
:10625000541D002070B50F4C052200212000FCF7D2
:106260009BFB0D4D2B78DA0707D50C4C9B070CD503
:106270000121200000F0B0FE70BD2000103000F0C1
:106280008BFE2B78054C9B07F2D4200000F084FE97
:10629000EEE7C046541D0020501D0020781D002050
:1062A000F0B54B79060083B0022B02D18B79022B1B
:1062B00003D00025280003B0F0BD204FBB78002B91
:1062C000F7D18B7809253B700C780C196378242B57
:1062D00007D00CE02378E4185D196378ADB2242B65
:1062E00005D19542F6D90020FFF766FEE2E71A00D5
:1062F000052B15D0042AF6D163790A2BF3D1104B64
:10630000277801930133009330000223E119023A08
:10631000FFF79EFC0028CCD00E35ED19ADB2E2E7B8
:1063200021003000FFF7E2FC0028C2D0A3787B7088
:1063300023785D19E4186278ADB2DBE7541D0020C4
:10634000561D0020F8B56023140012780500134094
:106350000020202B07D1304A6379277916781B0259
:106360003B439E4200D0F8BD6378222B1AD007D859
:10637000202B34D0212BF6D101293ED00120F2E789
:10638000232BF0D1012940D00329F7D1234B002B37
:10639000F4D0E178A37809020020194300E000BF9F
:1063A0000120E0E7012930D00329E7D101252E00A3
:1063B000A378E478023924021C4314712640243265
:1063C0001000714000F008FE154B002BD6D062087B
:1063D000002031002A4000E000BF0120C3E701296E
:1063E0000BD00329CAD10F4B002BC7D00832002095
:1063F0001100FEF7ADFA0120B5E7072321002800C0
:10640000094AFFF7F1FC0120ADE721002800FFF762
:10641000D5FC0120A7E7C046541D00200000000065
:1064200000000000514900105C1D0020F0B54F46EF
:106430004646D646C0B5364D8046EA780C001F0069
:106440008A423CD0AB788B4210D00020E0BCBA46E8
:10645000B146A846F0BD2F4B002B04D02E4800F0CB
:10646000ADFB002851D00020FFF7A6FDAB78A3427A
:1064700001D00120EAE7294B002B02D0002000E0E8
:1064800000BF0020FFF732FE0028F2D1244C20008C
:1064900000F07EFB0028ECD1002FEAD0BF06E8D147
:1064A000243C4046A178FFF73BFC0028E1D00023C4
:1064B00000224046A178FFF75BFC0120C6E79AB2B4
:1064C00010239A46174EAA443100504600F0A8FC0B
:1064D000154B002BBFD06B79FF2BBCD0002FBAD04F
:1064E000F219914603E001364E45B4D06B7932780B
:1064F0009A42F8D1504600F061FB0028F3D1534690
:10650000103B597900E000BFEDE700E000BFAAE7CB
:10651000541D002000000000641D00200000000049
:10652000781D0020D01C0020000000009322F0B550
:10653000134C85B0002120009200FCF72DFA2300B7
:106540002000802640270F4D4D337600FF33293041
:106550000295009300220023002103970196FF304B
:1065600000F0D4F94035201D2834002301220021F9
:10657000039702950196009400F0C8F905B0F0BDAC
:1065800018200020981F002010B5054C200000F0B6
:10659000F3F920002538FF3800F0EEF9012010BD96
:1065A0004021002070B5084C002520003130FF301C
:1065B000257000F0F1FC20000C3000F0EDFC2A23E7
:1065C000FF33E554657170BD18200020F8B55746BB
:1065D0004546DE464E46E0B54B7980460F00FF2B20
:1065E0005BD1404B99462A234946FF33CB5C002BB5
:1065F00053D14E79002E50D1BB783C780B703B794B
:106600003C19002B46D098235B004B449A460C2340
:106610004B449B46A51803E0AC423BD22378E418D8
:106620006378052BF8D1AC4234D221004046FFF705
:106630005DFB002831D0A3780136F6B2DB09012BCF
:1066400032D0504600F0A8FC2A234946A278FF33F6
:10665000CA54637922791B021343234A5B0594468B
:106660005B0D942163445A4253414A46022049003B
:10667000525C5B00824313434A46535451464046A2
:10668000083900F0E3F9002807D02378E4183B79B3
:10669000B342C5D8E01B80B200E00020F0BCBB468E
:1066A000B246A946A046F8BD584600F075FC5A46C9
:1066B000A3780C3A5371637921791B020B430A4981
:1066C0005B058C465B0D634459424B4102201179B6
:1066D0005B0081430B43594600200839137100F0D9
:1066E00081F9D2E71820002000FEFFFFF8B52A2527
:1066F00006001F48FF35455D1F008D4215D04379C8
:106700008B4201D00020F8BD1A4B002B04D0390475
:106710000020090C00E000BF174C3000210000F001
:1067200061F900281DD00120EDE79A235B00C35AD0
:10673000002B0DD1114B002B04D000201049BAB210
:1067400000E000BF30000F4900F080F90120DAE7D7
:1067500096235B00C1583130BAB2FF3000F060FBC5
:10676000E8E73A002100300000F008F90120CAE70C
:1067700018200020000000001C2000200000000065
:10678000981F00204021002000B5030083B000299D
:1067900010D00020012B07D80A78002A04D00C481A
:1067A000C2540120012A01D003B000BD1800FEF739
:1067B000D5FDF9E701236A46002001A99380FEF781
:1067C000CDFD0028F0D00122014B1A70ECE7C04645
:1067D000701E0020037870B5DB0704000E00DD0F8B
:1067E000002B17D103785B0701D5280070BD01216C
:1067F0003000494201F044FC2378DB07DD0F002B19
:106800000AD123785B0708D4042223780125134397
:10681000237002E00025E8E70025300001F008FCC5
:10682000E3E7C04670B50C00012106004942200094
:1068300001F026FC33785B07DD0F002B04DB200022
:1068400001F0F6FB280070BD3378DB0704D4042286
:10685000337893433370F2E70025F0E74379027908
:106860001B021343C2785B0592075B0D920F022A4D
:106870001DD0032A0CD00020012A08D102394A4237
:106880005141124A9446614499424041C0B2704716
:1068900002394A1E91410E4A494211408022D200DB
:1068A00094460020614499424041C0B2EFE702297A
:1068B00005D0002040229A424041C0B2E7E7054A95
:1068C000981843425841C0B2E1E7C046FF030000B8
:1068D00040FCFFFF00FEFFFF8A1870B5914207D20F
:1068E0007F264C78052C04D00C7809198A42F8D8F8
:1068F00070BD34008D782C4064000419ED09635597
:106900000C7809198A42ECD8F2E7C046F0B5C646C1
:1069100000B582B0150008AA40CA040017886A466C
:10692000928D012090460A00217802408143200088
:10693000114321703A00009331000123083000F028
:10694000F1F8002E01D0002F08D10A9B01206360CE
:106950004346638002B080BCB846F0BD26001C36BA
:106960003000FAF723F90023002D01D03300002670
:106970006361A661E9E7C04601207047F8B50224CB
:106980000B7807001C4063425C41144B64421C407E
:10699000134B08009C4608300D001600644400F0BC
:1069A000F7F8002807D1002E05D0344203D1012486
:1069B0002B781C4201D00020F8BD38006978FFF721
:1069C000AFF90028F7D02B781C42F4D10023002225
:1069D00038006978FFF7CCF9EEE7C04640FEFFFFCC
:1069E000FF010000F8B50D000835060028000C0076
:1069F00000F0CEF8002803D0012723781F4201D0F1
:106A00000020F8BD30006178FFF78AF90028F7D040
:106A100028006288616800F03DF9237805001F4076
:106A200000280BD0002FEBD10300626830006178A2
:106A3000FFF79EF90028E3D02800E2E7002FDFD11E
:106A400030006178FFF780F9DAE7C046F8B5CE4646
:106A5000474680B58A8906000C000B78002A07D1CA
:106A600001251D4240D00020C0BCB946B046F8BD4B
:106A70009B0733D42A4B4025994627000837380016
:106A800000F0A4F88542EED80122237890461A42FD
:106A9000E9D130006178FFF743F90028E3D03800EE
:106AA00000F094F8424623781A40854231D8002AF3
:106AB000D9D14A46638802401D1C934200D9151C57
:106AC000ADB200226178002D00D062682B0030004A
:106AD000FFF74EF90028C6D02800C5E7FE23802521
:106AE0001B029946AD00C8E74978FFF719F900285D
:106AF000B9D023781D42B6D1638800226178002B7B
:106B000000D062683000FFF733F90028ABD060880E
:106B1000AAE7002AA7D130006178FFF715F9A2E7AC
:106B2000C0FF0000F0B5C64600B504006846057E0B
:106B30008020884617001E000002824226D8E068A6
:106B4000002803D00121494201F09AFA2069002867
:106B500003D00121494201F093FA434623607304B4
:106B60005B0CED031D430023E0686381A780E58093
:106B70002381002801D001F05BFA2069002801D0B0
:106B800001F056FA012080BCB846F0BD0020FAE7BB
:106B900010B5048941898288A3B288B28C4207D398
:106BA0001B1A9BB2101C9A4200D9181C80B210BD4F
:106BB0005100091A5B189BB2F4E7C046038940896B
:106BC000181A43425841C0B27047C04610B50489F4
:106BD00041898288A3B288B28C4207D31B1A9BB228
:106BE00000209A4201D9D21A90B210BD5100091A60
:106BF0005B189BB2F4E7C04670B5040000690E0054
:106C0000002803D00121494201F03AFA2589608920
:106C1000A288A9B283B2854232D3CD1AADB2002D7B
:106C200028D0AA4208D291422FD3891A8BB263810D
:106C30009A4203D89B1A9BB29A42FBD9E2882168F8
:106C40005204520C53433000C918FBF7ABFE638962
:106C50000125591C89B2A2888B420DD9002152000E
:106C6000891A89B220696181002801D001F0E0F918
:106C7000280070BD618989B252009142F2DBEFE7D2
:106C80005500ED1A4D19ADB2C9E789188BB2638171
:106C9000CEE7C046F0B546464F46D646C0B50600DC
:106CA000006989469046002803D00121494201F03D
:106CB000E7F931897289B5888BB294B2914254D385
:106CC0001F1BBFB2002F4AD0BD4205D2AB4251D2EA
:106CD0005B199CB22F0074814346B8453DD89FB2E2
:106CE000A54203D8641BA4B2A542FBD9F28831683F
:106CF0005204520C904662432B1B9BB289184246A9
:106D00009F4225D953439BB21A0048469A46FBF747
:106D100049FE434648467D1B64195C433168504434
:106D2000A2B2FBF73FFE7189B588CB199BB26A000E
:106D3000994216D99B1A9BB230697381002801D001
:106D400001F076F93800E0BCBA46B146A846F0BD7D
:106D500048467A43FBF726FEE5E73B1CBFE773890D
:106D60009BB26A009342E7DBE4E76F003F1BDF1949
:106D7000BFB2A7E75B1B9CB2ACE7C046F8B5040006
:106D8000C0680E00002803D00121494201F078F9C3
:106D9000258920896189A288ADB283B28FB28842E9
:106DA00029D3DB1B9BB29A4209D8E779FF0906D1A8
:106DB000E068002801D001F03BF93800F8BD2B0055
:106DC00095421DD39B1A9BB29342FBD2E288206866
:106DD0005204520C53433100C018FBF7E3FD6B1C07
:106DE0009BB2A2889D4217D9002352009B1A9BB2E6
:106DF00001272381DCE75100C91B5B189BB2D2E756
:106E0000E28820685204520C53433100C018FBF74B
:106E1000C9FD0135A288ABB252009342E8DBE5E739
:106E2000F0B54E465746DE464546E0B58946060073
:106E3000170083B0002A67D0C068002803D0012162
:106E4000494201F01DF93389F2799BB29846738962
:106E5000B5889BB2D20940D198455ED26A00D31A58
:106E600043449BB2AB425DD2EB1A1A1C9BB2BB42AD
:106E700000D93A1C97B27B1B9BB20193F3885B0449
:106E80005B0C9A464346DB199BB29B464446A84599
:106E900003D3641BA4B2AC42FBD2534663433068B5
:106EA0002D1BADB2C018BD424BD3524649467A4362
:106EB000FBF778FDB3885B00D84501D89B4503DB21
:106EC0005A46D31A9BB29B465B463D003381F0681D
:106ED00000281AD001F0ACF817E0F2885204520CE6
:106EE0009246AF4220D298454DD34246D21A92B232
:106EF0006900781B80B2D21901908A4233DA434686
:106F0000FB189BB29B46C1E70025280003B0F0BCEC
:106F1000BB46B246A946A046F0BD4246D31A9BB234
:106F2000AB42A1D30025D2E7002DD0D07F1B574321
:106F300098465A19002392B2B94493462F00019300
:106F4000A4E753465D43ADB22A004946FBF72AFD4C
:106F5000019B2900E21853465A43306892B24944D3
:106F6000FBF720FDA6E75A1992B29346D21B92B2C4
:106F7000904693420CD94346591A8BB29846FB1857
:106F80009BB29B4682E76900CA1A424492B2B0E7BC
:106F9000914200DD7AE7EEE710B50400C0680028F2
:106FA00003D00121494201F06BF82069002803D089
:106FB0000121494201F064F80023E06863812381E4
:106FC000002801D001F034F82069002801D001F038
:106FD0002FF8012010BDC04670B50400C0680D0038
:106FE000002803D00121494201F04AF82069002815
:106FF00003D00121494201F043F87F21E379ED01FB
:107000001940E0682943E171002801D001F010F82F
:107010002069002801D001F00BF8012070BDC046A6
:1070200010B583070AD00300032102E001330B42AD
:1070300005D01A78002AF9D1181A10BD0300196872
:107040000C4A0D4C8A188A4322420FD15968094ACA
:1070500004338A188A43224208D15968054A043306
:107060008A188A432242F1D000E001331A78002ABC
:10707000FBD1E1E7FFFEFEFE8080808070B5074C0B
:10708000074D641BA41005D0013CA300EB589847A2
:10709000002CF9D100F0C0FF70BDC046288100105F
:1070A000288100100020704710B5034A03490448A6
:1070B00000F0ECFE10BDC046F0110020FD72001083
:1070C000B010002041680B4B10B50400994201D06C
:1070D00000F014F9A168084B994202D0200000F09A
:1070E0000DF9E168054B994202D0200000F006F945
:1070F00010BDC046C8190020301A0020981A002080
:1071000000207047F8B5CE464746344C344B354ADC
:107110002000002580B51A600423082200215C307D
:1071200025606560A560656625616561A561E360B0
:10713000FBF732FC2C4B2000994623622B4B2C4F43
:1071400098466362CC23E5502A4B2B4E636780231D
:1071500008220021C430E550A762E662A566E56614
:107160002567A567E567E461FBF716FC2200842329
:107170006832E2504A460433E2504246200004336B
:10718000E2500433E7500433E6503C33E550043317
:10719000E5500433E550194A5C33E550583BE25062
:1071A0000433E5502D300433E55008220433002128
:1071B000FF30E550FBF7F0FB2200EC23D032E25029
:1071C0004A460433E25042460433E2500433E75067
:1071D0000433E650C0BCB946B046F8BDC81900201B
:1071E000C4190020A9700010217C00104D7C0010F3
:1071F0008D7C001009000100BD7C0010120002000F
:10720000F8B5244B07001B68002B3BD0224E736857
:10721000B468013B03D51BE06834013B18D30C2252
:10722000A55E002DF8D120001C4B08220021E36050
:1072300065662560A560656025616561A5615C3056
:10724000FBF7AAFB256365636564A5642000F8BDB0
:107250003568002D01D02E00D9E7D621380049002D
:1072600000F09EF8041E10D00423D02205602500F3
:1072700043600C300021A0605200FBF78DFB3460AE
:107280002E00C4E7FFF73EFFC0E70C2330603B60F1
:10729000DCE7C046C4190020F01100200100FFFF08
:1072A000436B10B5002B00D010BD044B4363044B5F
:1072B0001B68002BF8D1FFF725FFF5E7C57000101C
:1072C000C41900207047C0467047C04610B5002062
:1072D000024A034900F0DAFD10BDC046F01100205B
:1072E000A570001010B50020024A034900F0CEFD41
:1072F00010BDC046F01100200171001070B50600ED
:107300000C1E08D0002802D0436B002B3BD00C226F
:10731000A35E002B02D10025280070BD21003000A3
:1073200000F0D2FCE36A0500002B04D03000E169D4
:10733000984700281DDBA3891B061FD4216B002959
:1073400008D023004033994202D0300000F05AFBAD
:1073500000232363616C002904D0300000F052FB4D
:1073600000236364FFF7AEFF0023A381FFF7ACFFA8
:10737000D2E70125A3896D421B06DFD530002169C4
:1073800000F040FBDAE7FFF78BFFC0E710B5034BD7
:1073900001001868FFF7B2FF10BDC046A81000201A
:1073A000F0B54E464546DE465746E0B50D000B3576
:1073B000060085B0162D27D8102900D9DAE000F094
:1073C00011FC102518230221C74FFB181A005C6816
:1073D000083A944200D146E103226368A1689343CE
:1073E000E268CA6091600121E3185A6830000A43DC
:1073F0005A6000F0F9FB2000083005B0F0BCBB4635
:10740000B246A946A046F0BD07239D4300D5B1E092
:10741000A94200D9AEE000F0E5FBFC235B009D42F1
:1074200000D294E1690A00D1A8E0042900D94FE113
:1074300038239846A90988443931CB0008225242A2
:107440009446A94FFB189C446346DC68A44514D0BD
:10745000032399460B0061469C4607E0E068002A3A
:1074600000DBFAE0814200D1FBE004004A46636899
:1074700093435A1B0F2AF1DD41463A003C6908321A
:10748000944200D1D8E0032063688343581B0F283F
:1074900000DD60E13A617A610028A4DA7A689046FA
:1074A00080229200934200D3E3E0DA0858090123D6
:1074B0008340404618438046D300DB199A687860C1
:1074C000E360A2609C60D46001208B10984040452E
:1074D0005CD8434603420AD1032399434346400004
:1074E0000431034203D1400004310342FBD00323A3
:1074F000B3469C460E00B8460190F000404401009F
:10750000B246CB680BE064465A681F00A243DB68B2
:10751000541B0F2C00DDEDE0002C00DB07E199424D
:10752000F1D101239946CA44534608319B07E8D15B
:10753000032205E003680838013E834200D001E2DF
:107540003242F7D14346019A5B6893434246536007
:10755000019A520001929A4216D8002A06D113E0ED
:1075600004229146019ACA44520001921342F7D074
:107570005646C2E70C23002033603EE780233F22BB
:10758000402190469B0059E75E4647460322BC686F
:10759000636893439846AB4202D35A1B0F2A4EDCD2
:1075A000230043440293514B08209A461B68103332
:1075B0005B19019300F08CFC4D4903900B688B46DE
:1075C000013306D08446019B4242013B6344134091
:1075D00001933000019900F009FB0300814601335B
:1075E00000D1D6E0029B834200D9D0E053465A68CE
:1075F000019B51469C4662444A60029803990139B6
:10760000484500D0E3E04846084200D0DFE0B968D2
:107610004344894601210B4349464B605146C96AA0
:10762000914201D25146CA625146096B914201D240
:1076300051460A634C46AEE07B68984644E7012316
:1076400029001A431943651961603000BD606A6002
:1076500000F0CAFA20000830CFE6A268D06082604D
:10766000C1E6614609E7DC680231A34200D104E7C4
:10767000B2E65A0A042A00D882E0142A00D907E1A7
:1076800010005B3082465C32D200082040428446C3
:10769000BA189444624692680B308146944500D1F2
:1076A000DEE00800A2466146844602E0926891420C
:1076B00004D04C465068A0439842F7D8D36861463E
:1076C00054469C466346A260E3609C60D460FBE63F
:1076D00014296DD9542900D9E3E06E239846290B6B
:1076E00088446F31CB00A9E608120020001B00205F
:1076F00000120020BA46012051468446491905432C
:1077000050464560856847466046EB605E469D6032
:10771000534639617961204308374860CF603000B3
:107720008F609C5000F060FA5046083065E6BA461B
:1077300001205E465244516801435160BA683000EE
:10774000D3609A6000F050FA3800083055E62B00FC
:10775000E908083338E66119884601218C460D4353
:107760004146656039617961CA608A606246024358
:107770004A60E050300000F037FA200008303CE664
:107780009A091000393238308246D2007DE7BC4277
:1077900014D0BC686368032293435A1BAB4202D3E4
:1077A0000F2A00DD4BE7300000F01EFA002024E62F
:1077B0005B23984688445C31CB003FE653465A68C9
:1077C000019B9C46534662445A60039B591E5B468C
:1077D0001B68013370D04B4602981B1A9B18524607
:1077E000536007234A4648461A400292184240D046
:1077F0000398013384469B1A019A99444A440192A2
:1078000063440A409B1A194030008B4600F0EEF9A1
:10781000431C77D04B46C01A03005B440193534688
:107820005A6801205A445A604B464946BB60019B46
:1078300003434B60BC4200D1F0E643460F2B3FD9D7
:1078400007210C3B8B4361680140052019436160AF
:10785000E118486088600F2B49D84B465B68DDE62D
:107860005346981001238340404618438046786071
:1078700028E7019B039A4B440B40D31A1940300070
:107880008B4600F0B3F9431CC4D100239B46C6E7E6
:10789000542A17D81A0B10006F326E308246D2006D
:1078A000F3E6AA235B00994217D8DD3B9846E90B23
:1078B00088447831CB00C1E55B464A461A6090E7C0
:1078C000486070E7AA204000824226D8DA0B1000F8
:1078D000783277308246D200D7E61C4B994226D8C0
:1078E0007C239846A90C88447D31CB00A6E5210075
:1078F0003000083100F086F853465A68BB68994654
:107900005B688BE6019A029B94464A46083B6344B7
:107910009B1A019300239B4681E70C4882420CD8B6
:107920009A0C10007D327C308246D200ADE6FE23F8
:107930007E227F2190469B0080E5FE227E209200E1
:107940008246A2E643465B6802E6C0465405000054
:10795000F0B5C646060000B508200D0000F0B8FAE4
:107960000400300000F03EF9234B210098469B684C
:107970005F6803239F4338001138401B0019FAF752
:10798000EDF8451E6543AC4208DC0021300000F0F4
:107990002DF943469B68DB19984206D0300000F071
:1079A00023F9002080BCB846F0BD3000694200F0E9
:1079B0001DF901300ED0012243467F1B9B681743FF
:1079C0000E4A5F60136830005B1B136000F00CF917
:1079D0000120E7E70021300000F008F943469A68EB
:1079E000831A0F2BDADD064C04492468001B08605B
:1079F00001210B435360D1E708120020041B002033
:107A000000120020F8B5CE46474605000C0080B5B0
:107A1000002957D000F0E6F8012321009C460839E0
:107A200048686246030003249343CF187A68654E82
:107A3000A243B468BC4200D170E0BC18A1466446C1
:107A40007A60044221D10868091A1B1888688046A8
:107A5000484640682040340008348146A04551D053
:107A60004046CC68C460A0604846002811D19B18ED
:107A70005548BA68824200D17FE0F868D0608260E1
:107A800001221A434A60CB5007E048464068204232
:107A9000EDD062461A434A603B60802292009342D6
:107AA00014D2DA08580901238340706803437360D5
:107AB000D3009B199A68CB608A609960D1602800D6
:107AC00000F092F8C0BCB946B046F8BD5C0A042C80
:107AD0003DD89C09200039343830E400341922683C
:107AE000083C0327944203D140E09268944203D0BB
:107AF0005068B8439842F8D8D468CC608A60A160D6
:107B0000D160DCE7002858D1B868D218FB68C360A0
:107B10009860634613434B608A50D0E79A186346D7
:107B2000034206D10B68C91A8868D218CB68C360B3
:107B30009860012313434B60244BB1601B68934250
:107B4000BDD8234B28001968FFF702FFB7E7142CB4
:107B500007D9542C1AD81C0B20006F346E30E40067
:107B6000BCE720005C345B30E400B7E70123801001
:107B70008340706803437360BFE7D1609160CA605F
:107B80008A6001221A434A60CB5098E7AA22520029
:107B9000944205D8DC0B200078347730E4009DE770
:107BA0000C4A944205D89C0C20007D347C30E400C3
:107BB00094E7FE247E20A40090E762461A434A60C0
:107BC0003B607CE708120020101200200412002005
:107BD000001B002054050000014B18687047C04688
:107BE000A81000207047C0467047C046002370B5FB
:107BF000064C050008002360FCF756FB431C00D030
:107C000070BD2368002BFBD02B60F9E7341B0020EC
:107C100010B5010000230022002000F0A1F910BDE2
:107C200070B50C000E25495F00F0D6F9002803DB83
:107C3000236D1B18236570BDA389024A1340A381DD
:107C4000F9E7C046FFEFFFFF00207047F8B50C00D2
:107C50001F000C23C95E05001600CB050AD40A4B91
:107C6000320019402800A1810E23E15E3B0000F0A4
:107C70003DF9F8BD0E23E15E0022022300F05CF91D
:107C80000C23E15EEBE7C046FFEFFFFF70B50C0091
:107C90000E25495F00F050F9431C07D08023A289CC
:107CA0005B0113431BB22065A38170BDA389024A07
:107CB00013401BB2F8E7C046FFEFFFFF10B50E23DD
:107CC000C95E00F027F910BDF0B5C64600B50C221C
:107CD0008B5E07000C001A0751D480254A682D01DD
:107CE0001D438D81002A00DC6CE0A66A002E42D084
:107CF0003A68E169904600223A60DB0467D40022CA
:107D000001233800B0470200431C00D16EE00C2371
:107D1000E55EA66AE1696D0706D56368D21A236B32
:107D2000002B01D0E36BD21A00233800B047431C6C
:107D30004FD139680C22A35E1D2962D8324ACA404D
:107D4000D2075ED5314A1A40A281002262602269C0
:107D50002260DB0401D5002946D04346216B3B60FD
:107D6000002908D023004033994202D03800FFF7A1
:107D700049FE00232363002080BCB846F0BD0E6995
:107D8000002EF8D00D680022AD1B0E609B0700D1BD
:107D90004A69A260002D04DCEDE736182D1A002D8B
:107DA000E9DD636A3200984638002B00E169C0477C
:107DB0000028F2DC4022A38913431BB20120A381D7
:107DC0004042D9E7CA6B002A00DD8EE7D3E7226D77
:107DD000A1E70C22A35E0D4A1A40A2810022626034
:107DE00022692260DB04B8D52065B6E73B68002B2A
:107DF00000D18CE71D2B01D0162BDBD143463B6015
:107E0000B9E740221343D9E701004020FFF7FFFF05
:107E100070B504000D00002802D0436B002B09D080
:107E20000C22AB5E0020002B03D029002000FFF7BE
:107E30004BFF70BDFFF734FAF2E7C04670B5041E81
:107E400015D00E4B1D68002D02D06B6B002B0AD095
:107E50000C22A35E0020002B00D170BD2100280061
:107E6000FFF732FFF9E72800FFF71AFAF0E7044AB4
:107E70000449054800F00AF8EFE7C046A8100020C2
:107E8000F0110020117E0010B0100020F8B5474618
:107E9000CE46884680B58146170000267D68BC68BE
:107EA000013D0DD4A389012B07D90E22A35E013316
:107EB00003D021004846C04706436834013DF1D253
:107EC0003F68002FEAD13000C0BCB946B046F8BDCB
:107ED000802310B55B01082801D1180010BDFFF701
:107EE0007BFE16230360173BF7E7C04670B504001E
:107EF000080011001A000023054D2B60FCF700FA62
:107F0000431C00D070BD2B68002BFBD02360F9E729
:107F1000341B0020002370B5064C050008002360C8
:107F2000FCF700FA431C00D070BD2368002BFBD087
:107F30002B60F9E7341B002070B504000800110025
:107F40001A000023054D2B60FCF7F0F9431C00D00C
:107F500070BD2B68002BFBD02360F9E7341B002099
:107F6000F0B5C6461A4C00B52568002D2AD06C68BD
:107F70001F2C2ADC002808D10020631C0234A40036
:107F80006B60615180BCB846F0BD8827A600AE1971
:107F9000F2510137FF37BC460122AC446746A2408C
:107FA0003F68904617436246176084277F00F3516D
:107FB0000228E1D1280042468D30FF300368134388
:107FC0000360D9E7034D2560D1E701204042D9E79E
:107FD000C81C0020381B002070B5040008001100E8
:107FE0001A000023054D2B60FCF778F9431C00D0E4
:107FF00070BD2B68002BFBD02360F9E7341B0020F9
:10800000034B10B5002B02D00248FFF701FE10BD54
:10801000000000007D700010F8B5C04600000000B0
:1080200001B40248844601BC604700BF0103002040
:1080300001B40248844601BC604700BF250200200D
:1080400001B40248844601BC604700BF3D040020E3
:1080500001B40248844601BC604700BF5D0F0020A8
:1080600001B40248844601BC604700BF5D0F002098
:1080700001B40248844601BC604700BFC100002033
:1080800001B40248844601BC604700BF990100204A
:1080900001B40248844601BC604700BF01010020D2
:1080A00001B40248844601BC604700BFD10C0020E7
:1080B00001B40248844601BC604700BF190C00208F
:1080C00001B40248844601BC604700BF810C002017
:1080D00001B40248844601BC604700BF410C002047
:1080E000ED18001019190010FD1A00108929001050
:1080F000B9210010C9280010251A001035190010E8
:1081000055190010691900105D0B0010711900104D
:10811000290F0010B5180010910700100180001001
:08812000154E0010FD020010D5
:108128000A3E3D2053494D554C4154494F4E20502D
:108138004152414D4554455253203D3C00000000FA
:10814800673D2025660A583D20256620593D202593
:10815800662047524F554E445F593D2025660A56C2
:10816800454C5F583D20252E66202056454C5F59CA
:108178003D2025660A0A00000D5B252E3266735DD8
:1081880020583A20252E326620593A20252E32666C
:108198002056454C5F583A20252E32662056454CCD
:1081A8005F593A20252E3266000000000A0A3E3D3B
:1081B800204F626A65637420456E6420537461744D
:1081C80073203D3C00000000583A20252E32662CD2
:1081D80020593A20252E32662C2056454C5F583AB5
:1081E80020252E32662C2056454C5F593A20252EE4
:1081F80032662054494D453A2025660A00000000A1
:108208000A3D3D3D3D3D3D3D3D3D3D3D3D3D3D3DC9
:108218003D3D3D3D3D3D3D3D3D3D3D3D3D3D3D3D86
:108228003D3D3D3D3D3D3D3D3D00000042554753F0
:108238002D502D3020412D312D6920556E646572E9
:108248002D6465762050726F746F00002D2D2D2DD2
:108258002D2D2D2D2D2D2D2D2D2D2D2D2D2D2D2D46
:108268002D2D2D2D2D2D2D2D2D2D2D2D2D2D2D2D36
:108278002D2D2D2D000000005B315D205068797395
:108288006963732073696D756C6174696F6E000042
:108298005B325D204E6F7468696E672100000000D4
:1082A8005B685D2048656C70000000005B635D20C2
:1082B80043726564697473005B785D2045786974FE
:1082C80000000000507265737320616E79206B6541
:1082D8007920746F20636F6E74696E75652E2E2E0B
:1082E800000000004E6F7468696E672068657265EB
:1082F800210000004E6F2068656C70206973207043
:10830800726F7669646564210000000050374D4A39
:10831800206F726967696E616C2100000A54686594
:108328002073797374656D20686173206265656E6A
:108338002068616C7465642E20506C6561736520DB
:10834800756E706C75672074686520706F776572DC
:1083580020736F757263652E2E2E0000496E76614C
:108368006C6964206F7074696F6E3A2025630A0027
:108378000A2A2A2A2050414E4943202A2A2A0A003A
:108388000A0000004E6F207370696E6C6F636B7328
:108398002061726520617661696C61626C650000BC
:1083A8004E6F207573657220495251732061726552
:1083B80020617661696C61626C6500004861726475
:1083C8007761726520616C61726D20256420616C33
:1083D800726561647920636C61696D656400000091
:1083E80048617264206173736572740052656C65CC
:1083F80061736500626F6F74325F77323571303840
:1084080030000000322E322E300000007069636F99
:10841800000000007069636F5F646576000000000B
:108428004A756E203137203230323600666E692B3D
:1084380000000000666E69006E616E00666E692D50
:108448000000000055534220737464696E202F2089
:108458007374646F75740000526173706265727230
:1084680079205069000000005069636F0000000027
:10847800426F617264204344430000005265736593
:1084880074000000556E68616E646C656420495222
:108498005120307825780A00657020253032582020
:1084A80077617320616C72656164792061766169B6
:1084B8006C61626C6500000043616E277420636F15
:1084C8006E74696E75652078666572206F6E2069B6
:1084D8006E616374697665206570202530325800B6
:1084E800FFFFFFFFFFFFFF7F06005250D3F07542EA
:1084F800F483001006005250E182887FFC8300104C
:1085080006005250ABB360530C8400100600525062
:10851800BBFF3CB61484001006005250861C0302B0
:108528001C840010060052505422A29D288400107A
:1085380005005250DE65F468149F0010483700109B
:10854800F8360010F836001040370010F8360010E2
:10855800F8360010F8360010F8360010F83600101B
:10856800F8360010F836001038370010F8360010CA
:1085780030370010F8360010F83600102837001091
:10858800683900105E370010583900105E37001047
:10859800423900105E3700105E3700105E37001059
:1085A8005E3700105E3700105E3700105E3700102F
:1085B800503700105E3700105E3700105E3700102D
:1085C8005E3700105E37001050370010063A001072
:1085D800B2360010B2360010B2360010B2360010B3
:1085E800B2360010B2360010B2360010B2360010A3
:1085F800B2360010B2360010B2360010B236001093
:10860800B2360010B2360010B2360010B236001082
:10861800B2360010B2360010B2360010B236001072
:10862800B2360010B2360010B2360010B236001062
:10863800B2360010B2360010B2360010B236001052
:10864800B2360010B2360010B23600107C39001075
:10865800D43900107C390010B2360010B236001040
:10866800B2360010B2360010B2360010B236001022
:10867800B2360010B2360010B2360010B236001012
:10868800B2360010B2360010B2360010B236001002
:10869800B2360010B2360010163C0010B236001088
:1086A800B2360010B2360010B2360010B2360010E2
:1086B800B2360010B2360010B2360010B2360010D2
:1086C800163C0010183A0010163C00107C390010B7
:1086D800D43900107C390010000000000000F03F81
:1086E8000000000000002440000000000000594085
:1086F8000000000000408F40000000000088C340D8
:1087080000000000006AF8400000000080842E414C
:1087180000000000D01263410000000084D7974198
:108728000000000065CDCD410D0A000000000000EA
:1087380079480010000000007D48001089480010AA
:10874800B5480010B1480010000000000A00000001
:1087580000000306A6000800020002009C001400A6
:10876800030057494E555342000000000000000026
:108778000000800004000100280044006500760025
:1087880069006300650049006E00740065007200AE
:108798006600610063006500470055004900440019
:1087A80000004E007B006200630037003300390090
:1087B8003800630031002D00370033006300640087
:1087C8002D0034006300620037002D0039003800A6
:1087D800620038002D003900310033006100380094
:1087E80066006300610037006200660036007D00A5
:1087F80000000000050F2100011C100500DF60DDEE
:10880800D88945C74C9CD2659D9E648A9F00000309
:1088180006A60001000000000600525053B4F4A15F
:108828004C84001000000000608400107084001068
:108838001028002078840010848400100902540055
:10884800030100807D080B000202020000090400F9
:108858000001020200040524002001052401000192
:1088680004240206052406000107058103080010F8
:1088780009040100020A0000000705020240000086
:10888800070582024000000904020000FF000105FC
:1088980012011002EF0201408A2E0A0000010102B3
:1088A800030100007C540010E455001034560010F9
:1088B800BC550010CE550010AC5500101C550010CA
:1088C800C8540010BC5400109E5900108459001060
:1088D80054570010BE590010545700106C5900101E
:1088E8005859001054570010445900104A580010A5
:1088F800545700102A5C00101C5C0010105C00101B
:108908005457001054570010FA5B00101C5C0010FC
:108918005457001054570010545700105457001063
:10892800545700105457001054570010B05B0010F3
:108938009E0D00209E0D0020E80D0020080E00204E
:108948004C0E00205E0E0020940D00200000000058
:10895800B56100102562001055620010A162001078
:10896800456300102D6400100000000000000000A6
:108978002D65001089650010A5650010CD650010F3
:0C89880011490010ED6600100000000016
:10899400F0840010FC840010088500101485001079
:1089A400208500102C8500103885001020880010C8
:1089B40003000068EFF3108C72B60268002AFCD042
:1089C400BFF35F8F04229A56002A0BDB002900D0E4
:1089D4000A6000201B68BFF35F8F00221A608CF3CB
:1089E40010887047D0221206126801201A71F1E72C
:1089F400F0B5C646150000B504001E000268EFF38A
:108A0400108172B61368002BFCD0BFF35F8F042370
:108A1400E3562268002B2BDBBFF35F8F002010602E
:108A240081F31088D02212061278002752B29046A1
:108A34009A420ED1002080BCB846F0BDBFF35F8FD0
:108A4400176081F310882800310000F029FF002806
:108A5400F0D12268EFF3108172B61368002BFCD0BA
:108A6400BFF35F8F237922687F2BE7D9434602E067
:108A7400D0231B061B682371BFF35F8F0023136091
:108A840081F310880120D6E7F0B5C64600B50D0085
:108A9400040000F015FFFA2206000F00002328004E
:108AA4000021920000F0F4FE36184F41002F02DA44
:108AB4000126174F7642D0231B061B6800259846D3
:108AC4000AE0BFF35F8F156081F31088300039002E
:108AD40000F0E6FE002818D12268EFF3108172B688
:108AE4001368002BFCD0BFF35F8F237922687F2BA0
:108AF400E7D943462371BFF35F8F0023136081F3EB
:108B04001088012080BCB846F0BD0020FAE7C046BA
:108B1400FFFFFF7F0268EFF3108172B61368002B2A
:108B2400FCD0BFF35F8FFF2303710368BFF35F8F34
:108B340000221A6081F3108840BF704710B5084CBA
:108B44002378002B0AD18023064807495B051A685D
:108B5400C25004338B42FAD10123237010BDC046A6
:108B640024280020642200100001001010B5014BDD
:108B7400984710BD65220020064B5A6802609A6827
:108B84004260DA6882601A69C2605A6902619B694C
:108B940043617047000002400268064B5A60426815
:108BA4009A608268DA60C2681A6102695A6142692D
:108BB4009A61704700000240034B1A68C0239B006F
:108BC4009343024A136070470C8001400C900140AB
:108BD400054B1A6880239B005340C0229200134027
:108BE400024A13607047C0460C8001400C9001405B
:108BF4000023F0B5DE4657464E4645469A46E0B554
:108C040089B001900E00988A45491B8B140098473F
:108C1400534681464349988A1B8B98475346424999
:108C24000500988A1B8B98478046FFF787FF02A8A8
:108C3400FFF7A2FFC847A847FFF7CAFF251E22D0A7
:108C44000823C0219C460220490562468B6A1A40CB
:108C540018423FD0631B002D2FD1002A11D1002CC4
:108C640011D0C0235B059B4602239A4606339946DE
:108C74005B464A4657469B6A1A401F4242D0002A26
:108C8400F6D0002C30D1FFF797FFC047FFF76EFFF7
:108C940002A8FFF781FF09B0F0BCBB46B246A94663
:108CA400A046F0BD002C2FD1C0225205926A9146F5
:108CB40008224F463A40BF072DD50D2B1BD9002A59
:108CC400F0D1C0225205926A914608224F463A409A
:108CD400BF07F2D4002A04D12B002343002BB4D1C4
:108CE400D1E72B00002CF9D00B6E013C337023002C
:108CF40001362B43F2E7019F013D3B7801370B66B8
:108D04000197E7E70025E5E7C0235B051B6E013CFF
:108D14003370013699E72B00002ADFD1DCE7C04627
:108D24004946000045580000464300000022154B08
:108D340010B59A60DA601A615A619A61DA611A624E
:108D44005A629A62DA621A635A639A63DA631A6439
:108D54005A649A64DA641A655A659A65DA651A6619
:108D64005A669A66DA661A675A679A67DA67F03259
:108D740092000021044800F06BFD044B044A1A6081
:108D840010BDC0460000105014240020DC27002031
:108D940080011050F0B54E464546DE465746E0B5D4
:108DA400214B00249E6D012585B0002E22D01F4B3F
:108DB4009A46012399461E4B984601E0202C19D06F
:108DC4002A00230001342F003240E4B26D00002A4F
:108DD400F4D0524697654A465B085B0022409B18D4
:108DE4005B01434418009B4600F01EFC002808D198
:108DF400BE43E3D105B0F0BCBB46B246A946A0468B
:108E0400F0BD5B46E0219A78DB8A01A883600023E9
:108E1400C900018001210271437100F025FC58460C
:108E240000F0A0FBE4E7C0460000115000301150F0
:108E3400D42300209823F0B5C646C84A00B5D558B7
:108E440080232E009B02102484B01E401D4274D047
:108E5400C34BC44C9A6AC44B00261A603B23E35CA0
:108E6400022B00D14FE17B23E35C022B00D1F3E022
:108E7400BB23E35C022B00D1FAE0FB23E35C022B6F
:108E840000D101E13C23FF33E35C022B00D12DE14F
:108E94007C23FF33E35C022B00D10EE1BC23FF33C0
:108EA400E35C022B00D13FE1FC23FF33E35C022BA4
:108EB40000D1F5E0AD4BE35C022B00D174E1AC4B87
:108EC400E35C022B00D105E1AA4BE35C022B00D149
:108ED40075E1A94BE35C022B00D132E1A74BE35CC3
:108EE400022B00D1A0E1A64BE35C022B00D171E17F
:108EF400A44BE35C022B00D1A1E1A34BE35C022B66
:108F040000D17FE1002E08D1A04B1B78002B04D1A7
:108F140080219F4A90338902D150C02269468F4BE9
:108F240092009B6C80265B058A805B0D012101A861
:108F3400029300F099FB974CB602EB0600D57FE054
:108F440080235B021D4231D01E4301230224984634
:108F5400844FBB7E002B14D000F082FC012800D982
:108F640072E0C02200213800920100F001FB3800B9
:108F740000F0F8FA00F074FC012802D9844B5C6616
:108F84001C664346FB702037012C22D1C0236A465D
:108F9400DB009380804A02AB03CA03C3012101A80A
:108FA40000F062FB80227A4B92021A6580235B01F7
:108FB4001D4210D18023DB011D4223D180231B02DB
:108FC4001D422FD1AE4200D0C0E104B080BCB846EF
:108FD400F0BD0124BDE700241E43604B1C60FFF775
:108FE400A5FE80236A465B0093801472012101A8C8
:108FF40000F03AFB8022664B12031A658023DB01E2
:109004001D42DBD01E4380236A46DB00938001218E
:1090140001A800F029FB10225D4B1A6580231B0276
:109024001D42CFD01E43A0236A46DB00938001215A
:1090340001A800F019FB8022554B12011A65C1E703
:10904400FFF7A8FE26007BE7544B444A1C66536E88
:109054002340A342FBD184E77833E75C002F00D19F
:1090640006E70233E25C002A00D00DE13E00FFE691
:10907400B833E75C002F00D1FFE60233E25C002A3C
:1090840000D0F9E03E00F8E6F833E75C002F00D1A9
:10909400F8E60233E25C002A00D041E13E00F1E64A
:1090A400F933FF33E75C002F00D103E70233E25CBE
:1090B400002A00D02BE13E00FCE67933FF33E75C65
:1090C400002F00D1EAE60233E25C002A00D015E169
:1090D4003E00E3E6324BE75C002F00D1F4E60233B6
:1090E400E25C002A00D001E13E00EDE63933FF33B3
:1090F400E75C002F00D1CBE60233E25C002A00D00B
:10910400EBE03E00C4E63833E65C002E00D1AAE66C
:109114000233E25C002A00D1A5E6200000222030C0
:10912400E25400F04DFA9EE6B933FF33E75C002FBA
:1091340000D1B9E60233E25C002A00D0C4E03E006C
:10914400B2E6184BE75C002F00D1C7E60233E25CBD
:10915400002A00D0B0E03E00C0E6C0460000115036
:1091640000400540D4230020C82300203B02000017
:109174007B020000BB020000FB0200003B03000076
:109184007B030000BB030000FB0300002228002037
:109194000030115010000200000010500020115047
:1091A4007A020000FA0200006B4BE75C002F00D14A
:1091B40085E60233E25C002A76D13E007FE6674B07
:1091C400E75C002F00D184E60233E25C002A63D11D
:1091D4003E007EE6624BE75C002F00D188E6023356
:1091E400E25C002A00D0A3E05E4BE35C022B30D1AA
:1091F4005D4BE35C002B27D15C4BE35C022B00D07E
:109204008BE63E005A4BE35C002B00D17AE6FF2349
:109214009B00E25C002A00D17FE60022E2541C3B62
:10922400E01800F0CDF978E6524BE75C002F00D14E
:1092340059E60233E25C002A16D13E0053E64A4B5B
:10924400E35C002B00D158E6EF239B00E25C002A8C
:1092540075D1464BE35C022B00D05EE6444BE35CE5
:10926400002B00D159E6D2E70022E2541C3BE0185F
:1092740000F0A6F93E0036E620000022A030E254B9
:109284003E0000F09DF9F8E5200000226030E25431
:109294003E0000F095F9EBE50022E2541C3BE01897
:1092A40000F08EF93E0014E60022E2541C3BE01864
:1092B40000F086F93E0002E60022E2541C3BE0186E
:1092C40000F07EF93E0009E620000022A130FF30C4
:1092D400E2543E0000F074F9E6E52000002221305B
:1092E400FF30E2543E0000F06BF9D1E50022E25475
:1092F4001C3BE01800F064F93E00E5E52000002284
:109304006130FF30E2543E0000F05AF9C6E5200017
:109314000022E130FF30E2543E0000F051F9C9E58B
:1093240020000022E030E2543E0000F049F9A9E5B3
:109334000022E2541C3BE01800F042F954E70022FA
:10934400E2541C3BE01800F03BF982E731000A4884
:10935400694000F0ADFAC0463A020000BA020000CB
:109364007A030000BB030000BA030000FB03000003
:10937400FA0300003A0300008C840010F0B5C646DE
:1093840000B50200838A008B8C46011C984200D9E8
:10939400191CD47880252000461EB04189B2ED0006
:1093A4000D434003284301256C405B1AD470547864
:1093B4009BB29382002C31D16446D568A4014E1E21
:1093C4002D19B0461469002923D0062E32D92B005A
:1093D40023439B072ED1631CEB1A022B2AD90023AB
:1093E4008F08BF00E658EE5004339F42FAD143463B
:1093F400ED19DB1BE419B94209D026782E70002B35
:1094040005D066786E70012B01D0A378AB70146917
:10941400938A64181461802212021043002B02D133
:109424008023DB0118436346002B00D0000480BC7A
:10943400B846F0BD0023E65CEE5401339942FAD1FC
:10944400E5E7C0468368F0B51A680400002900D037
:10945400120C63789205900D002B08D1E38AC3188F
:10946400E382238B834201D90023A382F0BDE36806
:10947400890125695E18471E002822D0062F26D9A7
:1094840001315B18EB1A022B21D92B0033439B07C4
:109494001DD10023120E9200F158E95004339A4270
:1094A400FAD1BF1AAD18B618904209D032782A7092
:1094B400002F05D072786A70012F01D0B278AA709B
:1094C4002569E38A2D18C318E3822561C9E70022C0
:1094D400B35CAB5401329042FAD12569F1E7C0463E
:1094E40010B50400836800211B68FFF7ABFF6368B5
:1094F4001B685B0002D5238B834200D010BD012181
:109504002000FFF79FFFF9E7084A0300126C0020D0
:10951400920703D49A78D209012A00D07047D87EE2
:10952400023843425841C0B2F8E7C0460000115027
:1095340010B5FFF7E9FF00280CD00749074B8C460C
:10954400074A9B6A126863449B1A0020C6229A4207
:109554004041C0B210BDC046E0FCFFFF00400540E2
:10956400C823002000238376436103617047C0460B
:1095740010B58368002901D01C682140002A12D04C
:109584008024E400114322420DD01A6822420CD1F7
:10959400084A0A401A60084A126C920703D40C2342
:1095A400033BFDD28368196010BD8178034800F045
:1095B4007FF9C046FFFBFFFF00001150A08400109C
:1095C400436870B50021802504001E68FFF7D6FEAD
:1095D400124B6D011A6C0543A37892070ED55B06F6
:1095E4000ED00F4B1E4080239B053343626800213D
:1095F400136020002A00FFF7BBFF70BDDB09F0D029
:10960400A38A002BEDD001212000FFF7B7FEA02391
:10961400044ADB05324005431343E7E700001150D9
:10962400FFFFFFAFFFFFFFDF70B5857E0400002D55
:1096340014D0FFF755FFA38A002B01D1280070BD79
:109644002000FFF775FF002803D0012300252377AE
:10965400F4E72000FFF7B4FF0025EFE78178014825
:1096640000F026F9C0840010F0B5CE46474680B518
:10967400437805000E0085B0062B08D86C4A9B0081
:10968400D3589F466B4A13780133DBB213706A4B8D
:109694001C686269EFF3108172B61368002BFCD06A
:1096A400BFF35F8FA1612000290000F0E1F8626937
:1096B400A369BFF35F8F0021116083F31088002832
:1096C40004D105B0C0BCB946B046F0BD32006978DB
:1096D400287800F0D5F8F4E70121584B1A788A432A
:1096E4001A701A7801318A431A7000225A701A7853
:1096F40002318A431A70CAE75149524F8946524986
:109704000024002388463A7812E043461B6861012E
:109714005B18002B06D0DB69002B03D0696828781E
:1097240098473A780134E4B2511C2300A14217DB74
:10973400A242EAD89B1A5B014B44ECE73F4B1A78F0
:10974400D207BED504211A780A431A709FE73B4B0F
:109754001A78D207B5D504211A788A431A7096E785
:10976400364F3B785B072BD504223B78002193438B
:109774003B706B460632981D00F06AF82B7801ACFA
:109784002370052363702C4B1B6898465A69EFF3CA
:10979400108172B61368002BFCD0BFF35F8F434671
:1097A40040469961210000F063F843465A699B6979
:1097B400BFF35F8F0021116083F31088002831D13B
:1097C400FB78DB0700D47CE76B460A220021981D56
:1097D40000F03EF82B7801AC2370032363706B68B0
:1097E4006360154B1D686A69EFF3108172B61368E4
:1097F400002BFCD0BFF35F8FA9612800210000F08B
:1098040037F86A69AB69BFF35F8F0021116083F396
:109814001088002800D154E732006178207800F0E5
:109824002FF84EE732006178207800F029F8C7E776
:109834003889001023280020D41E00207C1E00201C
:109844005489001021280020CC1C00207047C046F9
:1098540001B40248844601BC604700BF9929001046
:1098640001B40248844601BC604700BF31060010C1
:1098740001B40248844601BC604700BF7D6D0010FE
:1098840001B40248844601BC604700BF1D53001068
:1098940001B40248844601BC604700BF1928001087
:1098A40001B40248844601BC604700BF01130010A4
:1098B40001B40248844601BC604700BF3D06001065
:1098C40001B40248844601BC604700BF3114001053
:1098D4001000000000000000000001000000000073
:1098E4000000000000000200000000000000000072
:1098F4000000030000000000000000000000FF0062
:109904000000000001B5486801318E4600477046EA
:1099140009380149884701BD6D0A001000000000A4
:109924000000000000000000000000000000000033
:1099340020160020000000000000000000000000CD
:10994400503300004C330000543300005233000005
:109954004D5300004D4300005334000043340000D5
:10996400DD4A0010914A0010054A00107D4900109C
:109974000000000000010000D81E002010000C00B0
:1099840000000000000000000000000000000000D3
:1099940000000000FF000000B010002000000000E4
:1099A40000000000C8190020301A0020981A002076
:1099B40000000000000000000000000000000000A3
:1099C4000000000000000000000000000000000093
:1099D4000000000000000000000000000000000083
:1099E4000000000000000000000000000000000073
:1099F4000000000000000000000000000000000063
:109A04000000000000000000000000000000000052
:109A14000000000000000000000000000000000042
:109A24000000000000000000000000000000000032
:109A34000000000000000000010000000000000021
:109A44000E33CDAB34126DE6ECDE05000B000000E6
:109A54000000000000000000000000000000000002
:109A640000000000000000000000000000000000F2
:109A740000000000000000000000000000000000E2
:109A840000000000000000000000000000000000D2
:109A940000000000000000000000000000000000C2
:109AA40000000000000000000000000000000000B2
:109AB40000000000000000000000000000000000A2
:109AC4000000000000000000000000000000000092
:109AD4000000000000000000000000000000000082
:109AE4000000000003000000C8190020000000006E
:109AF400FFFFFFFF00000200000000000000000064
:109B04000812002008120020101200201012002059
:109B14001812002018120020201200202012002009
:109B240028120020281200203012002030120020B9
:109B34003812002038120020401200204012002069
:109B44004812002048120020501200205012002019
:109B540058120020581200206012002060120020C9
:109B64006812002068120020701200207012002079
:109B74007812002078120020801200208012002029
:109B840088120020881200209012002090120020D9
:109B94009812002098120020A0120020A012002089
:109BA400A8120020A8120020B0120020B012002039
:109BB400B8120020B8120020C0120020C0120020E9
:109BC400C8120020C8120020D0120020D012002099
:109BD400D8120020D8120020E0120020E012002049
:109BE400E8120020E8120020F0120020F0120020F9
:109BF400F8120020F81200200013002000130020A7
:109C04000813002008130020101300201013002054
:109C14001813002018130020201300202013002004
:109C240028130020281300203013002030130020B4
:109C34003813002038130020401300204013002064
:109C44004813002048130020501300205013002014
:109C540058130020581300206013002060130020C4
:109C64006813002068130020701300207013002074
:109C74007813002078130020801300208013002024
:109C840088130020881300209013002090130020D4
:109C94009813002098130020A0130020A013002084
:109CA400A8130020A8130020B0130020B013002034
:109CB400B8130020B8130020C0130020C0130020E4
:109CC400C8130020C8130020D0130020D013002094
:109CD400D8130020D8130020E0130020E013002044
:109CE400E8130020E8130020F0130020F0130020F4
:109CF400F8130020F81300200014002000140020A2
:109D0400081400200814002010140020101400204F
:109D140018140020181400202014002020140020FF
:109D240028140020281400203014002030140020AF
:109D3400381400203814002040140020401400205F
:109D4400481400204814002050140020501400200F
:109D540058140020581400206014002060140020BF
:109D6400681400206814002070140020701400206F
:109D7400781400207814002080140020801400201F
:109D840088140020881400209014002090140020CF
:109D94009814002098140020A0140020A01400207F
:109DA400A8140020A8140020B0140020B01400202F
:109DB400B8140020B8140020C0140020C0140020DF
:109DC400C8140020C8140020D0140020D01400208F
:109DD400D8140020D8140020E0140020E01400203F
:109DE400E8140020E8140020F0140020F0140020EF
:109DF400F8140020F814002000150020001500209D
:109E0400081500200815002010150020101500204A
:109E140018150020181500202015002020150020FA
:109E240028150020281500203015002030150020AA
:109E3400381500203815002040150020401500205A
:109E4400481500204815002050150020501500200A
:109E540058150020581500206015002060150020BA
:109E6400681500206815002070150020701500206A
:109E7400781500207815002080150020801500201A
:109E840088150020881500209015002090150020CA
:109E94009815002098150020A0150020A01500207A
:109EA400A8150020A8150020B0150020B01500202A
:109EB400B8150020B8150020C0150020C0150020DA
:109EC400C8150020C8150020D0150020D01500208A
:109ED400D8150020D8150020E0150020E01500203A
:109EE400E8150020E8150020F0150020F0150020EA
:109EF400F8150020F8150020001600200016002098
:109F0400000000000000000000000000000000004D
:04000005100001E9FD
:00000001FF
